:100000006F006047130000001300000013000000A1
:100010001300000013000000130000001300000094
:100020001300000013000000130000001300000084
:08003000130000007300100032
:100038000000000000000000280200003802000054
:1000480000000000000400000000000000000000A4
:10005800020400000404000000000000000000008A
:10006800522C0000000000000804000000000000FE
:100078000A0400000C0400000E0400001004000034
:100088001204000014040000160400001804000004
:100098001A0400001C0400001E040000883100003F
:1000A80022040000240400002604000028040000A4
:1000B8002A0400002C040000543100003004000021
:1000C8003204000034040000360400003804000044
:1000D8003A0400002C3F00003E04000040040000E9
:1000E80042040000440400004604000048040000E4
:1000F8004A0400004C0400004E04000050040000B4
:1001080052040000364D00004C4D0000624D0000C6
:100118005A0400005C0400005E0400006004000053
:100128006204000064040000660400006804000023
:100138006A040000743F00006E04000070040000B0
:1001480072040000740400000000000000000000B9
:100158000000000000000000000000000000000097
:100168000000000000000000000000000000000087
:0801780000000000000000007F
:100180003D432A876373C3029377F700BDEFADE564
:10019000937606FF3D8ABA960CC34CC30CC74CC776
:1001A0004107E36BD7FE11E28280B306C3408A06A3
:1001B0009702000096966780A6002307B700A30663
:1001C000B7002306B700A305B7002305B700A304B3
:1001D000B7002304B700A303B7002303B700A302AB
:1001E000B7002302B700A301B7002301B700A300A3
:1001F000B7002300B700828093F5F50F9396850032
:10020000D58D93960501D58D61B7939627009702FA
:10021000000096968682E78086FA9680C1171D8F29
:100220003E96E374C3F8A5B7411122C60008010049
:100230003244410173002030411122C6000801A060
:10024000411106C622C400080945EF10A058EF501E
:10025000A024EF50002C01A0411106C622C40008C2
:10026000B71702409843B71702401367170098C3A7
:10027000B7170240D443B71702403707FFF8758F0E
:10028000D8C3B71702409443B71702403707F7FEA9
:100290007D17758F98C3B71702409443B717024074
:1002A0003707FCFF7D17758F98C3B7170240D443FB
:1002B000B7170240370781FF7D17758FD8C3B7176F
:1002C000024037079F0098C731200100B240224406
:1002D00041018280411106C622C40008312001007C
:1002E000B240224441018280011122CE0010232617
:1002F00004FE232404FEB71702409443B7170240BC
:100300004167558F98C3B71702409843B70702005B
:10031000F98F2324F4FE8327C4FE85072326F4FEE9
:10032000832784FE91E70327C4FE8567E31DF7FC5E
:10033000B71702409843B7070200F98F89C785476E
:100340002324F4FE19A0232404FE032784FE8547FA
:100350006312F70A37170240B71702405843D8C351
:1003600037170240B71702405843D8C3B7170240A7
:10037000D843B717024013670740D8C3B7170240E6
:10038000D443B71702403707C1FF7D17758FD8C315
:10039000B7170240D443B717024037072900558FDB
:1003A000D8C3B71702409443B7170240370700017C
:1003B000558F98C30100B71702409843B707000252
:1003C000F98FF5DBB7170240D843B7170240719B8E
:1003D000D8C3B7170240D843B717024013672700A6
:1003E000D8C30100B7170240DC4313F7C700A14789
:1003F000E31AF7FE010072440561828001A001A0AA
:1004000001A001A001A001A001A001A001A001A0E4
:1004100001A001A001A001A001A001A001A001A0D4
:1004200001A001A001A001A001A001A001A001A0C4
:1004300001A001A001A001A001A001A001A001A0B4
:1004400001A001A001A001A001A001A001A001A0A4
:1004500001A001A001A001A001A001A001A001A094
:1004600001A001A001A001A001A001A001A001A084
:1004700001A001A001A0970100209381A15617813E
:100480000020130121B817D500001305E59097054A
:100490000020938525B71386818163FAC5008322E6
:1004A000050023A0550011059105E3EAC5FE13855B
:1004B00081819385C1CE6377B500232005001105A6
:1004C000E36DB5FEFD42739002BC8D427390428095
:1004D0009302800873A0023097020000938202B654
:1004E00093E2320073905230EFF01FD79702000072
:1004F000938242D57390123473002030011106CEDE
:1005000022CC00102326A4FE0327C4FEB7270140F7
:1005100093870740631DF700854513050020EF1002
:100520003005814513050020EF1090041DA003271E
:10053000C4FEB737014093870780631CF7008545E9
:1005400013050040EF10D002814513050040EF1065
:1005500030020100F240624405618280797122D646
:100560000018232EA4FC232CB4FC232604FEA30590
:1005700004FE8327C4FDDC432326F4FE0327C4FEC8
:10058000B707F1E09387F7EFF98F2326F4FE83276F
:1005900084FD9843832784FD9C4F5D8F832784FDD2
:1005A000DC4F5D8F832784FDDC43A207D98F0327AF
:1005B000C4FED98F2326F4FE8327C4FD0327C4FE7F
:1005C000D8C38327C4FD9C472326F4FE0327C4FE1B
:1005D000B7F7F1FF9387D77FF98F2326F4FE8327A0
:1005E00084FD984B832784FDDC475D8F832784FD42
:1005F0009C478607D98F0327C4FED98F2326F4FE94
:100600008327C4FD0327C4FE98C78327C4FDDC5796
:100610002326F4FE0327C4FEB70710FFFD17F98F4A
:100620002326F4FE832784FDDC2BFD1713F7F70F39
:100630008347B4FED98FA305F4FE8347B4FED207E7
:100640000327C4FED98F2326F4FE8327C4FD032786
:10065000C4FED8D70100325445618280011122CEF8
:1006600000102326A4FE2324B4FE832784FE91CB0E
:100670008327C4FE9C4713E717008327C4FE98C74F
:1006800009A88327C4FE9C4713F7E7FF8327C4FE0E
:1006900098C70100724405618280011122CE0010CA
:1006A0002326A4FE2324B4FE832784FE91CB832734
:1006B000C4FE9C4713E707108327C4FE98C709A808
:1006C0008327C4FE9C4713F7F7EF8327C4FE98C720
:1006D0000100724405618280797122D60018232EB0
:1006E000A4FCAE87232AC4FC231DF4FCA30704FE4C
:1006F0008357A4FDA307F4FE832744FD99CB8327EA
:10070000C4FDD8438347F4FE5D8F8327C4FDD8C35F
:1007100021A88327C4FDD8438347F4FE93C7F7FF7E
:100720007D8F8327C4FDD8C3010032544561828088
:10073000011122CE00102326A4FE8327C4FE9C476D
:1007400013E787008327C4FE98C701007244056140
:100750008280797122D60018232EA4FC232604FE61
:100760008327C4FD9C47A18B89C785472326F4FEB8
:1007700019A0232604FE8327C4FE3E85325445611A
:100780008280011122CE00102326A4FE8327C4FEFE
:100790009C4713E747008327C4FE98C701007244B3
:1007A00005618280797122D60018232EA4FC2326AD
:1007B00004FE8327C4FD9C47918B89C78547232668
:1007C000F4FE19A0232604FE8327C4FE3E8532547E
:1007D00045618280011122CE00102326A4FE23242D
:1007E000B4FE832784FE99CB8327C4FE9847B707BE
:1007F00050005D8F8327C4FE98C719A88327C4FEC5
:100800009847B707B0FFFD177D8F8327C4FE98C7B1
:100810000100724405618280797122D60018232E6E
:10082000A4FCAE873687A30DF4FCB287230DF4FC3D
:10083000BA87A30CF4FC232604FE232404FE0347FA
:10084000B4FDA54763F6E7068327C4FDDC472326EE
:10085000F4FE8347B4FD138767FFBA878607BA970C
:100860001D47B317F7002324F4FE832784FE93C7A4
:10087000F7FF0327C4FEF98F2326F4FE834694FD79
:100880008347B4FD138767FFBA878607BA97B39784
:10089000F6002324F4FE0327C4FE832784FED98FA9
:1008A0002326F4FE8327C4FD0327C4FED8C785A0F2
:1008B0008327C4FD9C4B2326F4FE0347B4FDBA876F
:1008C0008607BA971D47B317F7002324F4FE832742
:1008D00084FE93C7F7FF0327C4FEF98F2326F4FE97
:1008E000834694FD0347B4FDBA878607BA97B3974A
:1008F000F6002324F4FE0327C4FE832784FED98F49
:100900002326F4FE8327C4FD0327C4FE98CB0347A8
:10091000A4FD994763E6E7068327C4FDDC5B232635
:10092000F4FE8347A4FD1387F7FFBA878A07BA97B7
:100930007D47B317F7002324F4FE832784FE93C773
:10094000F7FF0327C4FEF98F2326F4FE8346B4FD88
:100950008347A4FD1387F7FFBA878A07BA97B3972F
:10096000F6002324F4FE0327C4FE832784FED98FD8
:100970002326F4FE8327C4FD0327C4FED8DBE9A8A1
:100980000347A4FDB14763E6E7068327C4FD9C5BEC
:100990002326F4FE8347A4FD138797FFBA878A07AF
:1009A000BA977D47B317F7002324F4FE832784FE0C
:1009B00093C7F7FF0327C4FEF98F2326F4FE83466F
:1009C000B4FD8347A4FD138797FFBA878A07BA97B8
:1009D000B397F6002324F4FE0327C4FE832784FE86
:1009E000D98F2326F4FE8327C4FD0327C4FE98DB9A
:1009F000A5A08327C4FDDC572326F4FE8347A4FD6E
:100A0000138737FFBA878A07BA977D47B317F7006E
:100A10002324F4FE832784FE93C7F7FF0327C4FE35
:100A2000F98F2326F4FE8346B4FD8347A4FD138784
:100A300037FFBA878A07BA97B397F6002324F4FEE4
:100A40000327C4FE832784FED98F2326F4FE832741
:100A5000C4FD0327C4FED8D701003254456182800B
:100A6000797122D60018232EA4FCAE87231DF4FC36
:100A7000232604FE232404FE232204FE8357A4FD20
:100A8000A183C207C1832324F4FE8327C4FDDC4372
:100A90000357A4FD1377F70FF98F2322F4FE832762
:100AA000C4FD9843832784FEF98F81CB832744FEBE
:100AB00089C785472326F4FE19A0232604FE832731
:100AC000C4FE3E85325445618280797122D6001879
:100AD000232EA4FCAE87231DF4FCA30704FE83573A
:100AE000A4FDA183C207C183A307F4FE8347F4FEDC
:100AF00013C7F7FF8327C4FD98C301003254456133
:100B00008280011122CE00102326A4FE8327C4FE7A
:100B10009843C167F9177D8F8327C4FE98C3832745
:100B2000C4FE23A007008327C4FE23A20700832757
:100B3000C4FE23A407008327C4FE23A607000327BF
:100B4000C4FEB7070240A107631BF700B7070240C6
:100B5000D843B70702401367F700D8C3DDA80327BF
:100B6000C4FEB7070240F107631BF700B707024056
:100B7000D843B70702401367070FD8C3D9A8032784
:100B8000C4FEB707024093870703631DF700B7074A
:100B90000240D443B70702400567130707F0558F9B
:100BA000D8C345A80327C4FEB7070240938747046C
:100BB000631BF700B7070240D443B70702403D6705
:100BC000558FD8C379A00327C4FEB7070240938787
:100BD0008705631CF700B7070240D443B7070240FC
:100BE00037070F00558FD8C3ADA00327C4FEB70742
:100BF00002409387C706631CF700B7070240D4433F
:100C0000B70702403707F000558FD8C399A00327D4
:100C1000C4FEB707024093870708631CF700B707B5
:100C20000240D443B70702403707000F558FD8C39F
:100C30000DA00327C4FEB707024093874709631A34
:100C4000F700B7070240D843B70702401367F70021
:100C5000D8C30100724405618280797122D60018E0
:100C6000232EA4FC232CB4FC232604FE8327C4FDDE
:100C70009C432326F4FE0327C4FEE177BD07F98FCA
:100C80002326F4FE832784FD9847832784FD9C5305
:100C90005D8F832784FD9C4B5D8F832784FDDC4B18
:100CA0005D8F832784FD9C4F5D8F832784FDDC4F00
:100CB0005D8F832784FDDC535D8F832784FD9C57E4
:100CC000D98F0327C4FED98F2326F4FE8327C4FDC2
:100CD0000327C4FE98C3832784FDD8478327C4FD18
:100CE000D8C3832784FD98438327C4FD98C78327EF
:100CF00084FDD8438327C4FDD8C701003254456121
:100D00008280011122CE00102326A4FE2324B4FEEB
:100D1000832784FE91CB8327C4FE9C4313E71700EF
:100D20008327C4FE98C311A88327C4FE9843C167D4
:100D3000F9177D8F8327C4FE98C3010072440561B3
:100D40008280011122CE00102326A4FE2324B4FEAB
:100D50002322C4FE832744FE99CB8327C4FE9843F5
:100D6000832784FE5D8F8327C4FE98C321A8832731
:100D7000C4FE9843832784FE93C7F7FF7D8F8327A4
:100D8000C4FE98C30100724405618280797122D645
:100D90000018232EA4FC232604FE232404FEB707F8
:100DA00002409C432324F4FE032784FE8327C4FDD2
:100DB000F98F89C785472326F4FE19A0232604FE50
:100DC0008327C4FE3E85325445618280011122CEC4
:100DD00000102326A4FEB70702400327C4FED8C391
:100DE0000100724405618280397122DE8000232671
:100DF000A4FC2324B4FC232604FE232004FE232485
:100E000004FE232E04FC232204FE232C04FC83274F
:100E100084FC9C47BD8B2326F4FE832784FC9C47DF
:100E2000C18B89CB832784FCDC430327C4FED98F85
:100E30002326F4FE832784FC9E2393F7F70FE9CF44
:100E40008327C4FC9C432322F4FE232404FE5DA8D4
:100E5000832784FE0547B317F700232EF4FC83276E
:100E600084FC9E233E878327C4FDF98F2320F4FE54
:100E7000032704FE8327C4FD6311F708832784FE3C
:100E80008A07232EF4FC8327C4FD3D47B317F700E0
:100E9000232CF4FC832784FD93C7F7FF032744FE2C
:100EA000F98F2322F4FE8327C4FD0327C4FEB31762
:100EB000F700032744FED98F2322F4FE832784FC06
:100EC000984793078002631BF700832784FE05473A
:100ED0003317F7008327C4FCD8CB05A0832784FCF5
:100EE000984793078004631AF700832784FE054719
:100EF0003317F7008327C4FC98CB832784FE85072C
:100F00002324F4FE032784FE9D47E3F3E7F48327BD
:100F1000C4FC032744FE98C3832784FC9A239307C9
:100F2000F00F63F0E70E8327C4FCDC432322F4FEBA
:100F3000232404FE6DA8832784FEA1070547B31769
:100F4000F700232EF4FC832784FC9E233E8783270F
:100F5000C4FDF98F2320F4FE032704FE8327C4FD7C
:100F60006312F708832784FE8A07232EF4FC832765
:100F7000C4FD3D47B317F700232CF4FC832784FD01
:100F800093C7F7FF032744FEF98F2322F4FE83273C
:100F9000C4FD0327C4FEB317F700032744FED98F0F
:100FA0002322F4FE832784FC984793078002631B67
:100FB000F700832784FEA10705473317F70083272F
:100FC000C4FCD8CB832784FC984793078004631B19
:100FD000F700832784FEA10705473317F70083270F
:100FE000C4FC98CB832784FE85072324F4FE0327C3
:100FF00084FE9D47E3F1E7F48327C4FC032744FE06
:10100000D8C30100725421618280797122D6001800
:10101000232EA4FCAE87231DF4FCA30704FE832724
:10102000C4FD98478357A4FDF98F89C78547A30757
:10103000F4FE19A0A30704FE8347F4FE3E85325454
:1010400045618280011122CE00102326A4FEAE87C6
:101050002322C4FE2315F4FE832744FE99C70357B9
:10106000A4FE8327C4FE98CB31A00357A4FE832798
:10107000C4FED8CB0100724405618280797122D60A
:101080000018232EA4FC232CB4FC232404FE2322CA
:1010900004FE232604FE232004FE8327C4FD63D818
:1010A0000700B7070140DC4F2326F4FE31A0B70745
:1010B0000140DC432326F4FE8327C4FDC183BD8B9E
:1010C0002320F4FE0327C4FDC167FD17F98F2324F5
:1010D000F4FE8327C4FD63D407080327C4FDB707C4
:1010E00030007D8FB70730006314F702832704FEBA
:1010F000C1070D47B317F7002322F4FE832744FEF0
:1011000093C7F7FF0327C4FEF98F2326F4FEC5A873
:101110000327C4FDB7071000F98F95C3832704FE8A
:101120000D47B317F7002322F4FE832744FE93C72D
:10113000F7FF0327C4FEF98F2326F4FEC9A08327F7
:10114000C4FDD5839207032784FEB317F70093C726
:10115000F7FF0327C4FEF98F2326F4FE4DA00327D3
:10116000C4FDB70730007D8FB70730006315F70265
:101170000327C4FEB70700F1FD17F98F2326F4FEFD
:10118000B7070140D443B7070140370700F17D1787
:10119000758FD8C3ADA00327C4FDB7071000F98F22
:1011A0008DCB832704FE0D47B317F7002322F4FEEF
:1011B000832744FE93C7F7FF0327C4FEF98F232636
:1011C000F4FE0327C4FEB707000FD98F2326F4FED1
:1011D0003DA08327C4FDD5839207032784FEB31760
:1011E000F70093C7F7FF0327C4FEF98F2326F4FE09
:1011F0000327C4FEB707000FD98F2326F4FE8327E9
:1012000084FD91CF8327C4FDD5839207032784FEF5
:10121000B317F7000327C4FED98F2326F4FE8327D4
:10122000C4FD63D80700B70701400327C4FED8CF29
:1012300031A0B70701400327C4FED8C301003254D0
:1012400045618280397106DE22DC80002326A4FC01
:101250002324B4FC231704FE231504FE9147231610
:10126000F4FEB7177A00938707202322F4FE832722
:10127000C4FCDE232317F4FE8357E4FE93F707FC38
:101280002317F4FE930704FD3E85792F832784FD01
:101290002322F4FE032744FEB7470F009387072459
:1012A000B357F7022315F4FE0357E4FE8357A4FE59
:1012B000D98F2317F4FE8327C4FC0357E4FEDAA377
:1012C0008327C4FC9E23C207C183F99B13970701A0
:1012D00041838327C4FC9AA3231704FE832784FC3D
:1012E0009843E1679387076A63E5E704832784FCF3
:1012F0009C438607032744FEB357F7022316F4FEE8
:101300000357C4FE8D4763E5E70091472316F4FEBB
:101310000357E4FE8357C4FED98F2317F4FE835787
:10132000A4FE85071397070141838327C4FC9AB362
:1013300065A0832784FCFA23B167FD17631FF700BC
:10134000832784FC9843BA878607BA97032744FE0D
:10135000B357F7022316F4FE2DA0832784FC98438D
:10136000BA878607BA978E07BA97032744FEB35702
:10137000F7022316F4FE0357C4FE9167D98F231694
:10138000F4FE0357C4FE8567FD17F98F99E783576D
:10139000C4FE93E717002316F4FE0357C4FE8357D9
:1013A000E4FED98F139707014183E177D98F231783
:1013B000F4FE0357A4FE9307C0123307F702930706
:1013C000803EB347F702C207C18385071397070121
:1013D00041838327C4FC9AB38327C4FC0357E4FEEC
:1013E000DAAF8327C4FC9E23C207C18393E71700AB
:1013F0001397070141838327C4FC9AA38327C4FC66
:101400009E232317F4FE8357E4FE93F757BF231759
:10141000F4FE832784FCDA23832784FCBE27D98F3C
:101420001397070141838357E4FED98F2317F4FEF6
:101430008327C4FC0357E4FE9AA3832784FCDA279E
:10144000832784FC9E27D98F139707014183832725
:10145000C4FC9AA70100F2506254216182800111FC
:1014600022CE00102326A4FE2324B4FE832784FE6C
:1014700099CF8327C4FE9E23C207C18393E7170039
:101480001397070141838327C4FE9AA329A88327C2
:10149000C4FE9E23C207C183F99B139707014183B2
:1014A0008327C4FE9AA30100724405618280011162
:1014B00022CE00102326A4FE2324B4FE832784FE1C
:1014C00099CF8327C4FE9E23C207C18393E70710E9
:1014D0001397070141838327C4FE9AA331A883276A
:1014E000C4FE9E23C207C18393F7F7EF139707014A
:1014F00041838327C4FE9AA3010072440561828060
:10150000011122CE00102326A4FE2324B4FE83273B
:1015100084FE99CF8327C4FE9E23C207C18393E72D
:1015200007201397070141838327C4FE9AA331A89C
:101530008327C4FE9E23C207C18393F7F7DF139767
:10154000070141838327C4FE9AA301007244056109
:101550008280011122CE00102326A4FE2324B4FE93
:10156000832784FE99CF8327C4FE9E23C207C183AD
:1015700093E707401397070141838327C4FE9AA38B
:1015800031A88327C4FE9E23C207C18393F7F7BF08
:101590001397070141838327C4FE9AA30100724475
:1015A00005618280011122CE00102326A4FEAE87A1
:1015B000A305F4FE8347B4FE1397070141838327F5
:1015C000C4FE9AAB0100724405618280011122CEF3
:1015D00000102326A4FE8327C4FE9E2BC207C183CE
:1015E00093F7F70F3E85724405618280011122CE88
:1015F00000102326A4FEAE873287A305F4FEBA8727
:101600002305F4FE8347A4FE81CB8347B4FE93E712
:101610001700A305F4FE31A08347B4FEF99BA30590
:10162000F4FE8347B4FE1397070141838327C4FE6A
:101630009AAB0100724405618280797122D600184C
:10164000232EA4FC232CB4FC232404FE232204FE1A
:10165000232004FE232604FE8327C4FDDE2BC207BD
:10166000C1832322F4FE8327C4FD9E2FC207C183BA
:101670002320F4FE832704FEC2072320F4FE032761
:1016800044FE832704FE5D8FB7070001FD17F98F25
:101690002324F4FE032784FE832784FDF98F032788
:1016A00084FD6316F70085472326F4FE19A0232640
:1016B00004FE8327C4FE3E853254456182807971E1
:1016C00022D60018232EA4FC232CB4FC232604FECF
:1016D000232404FE232204FE8327C4FD2322F4FED8
:1016E000832784FDF1832324F4FE032784FDB707B9
:1016F0000001FD17F98F232CF4FC832784FE99C782
:10170000832744FED1072322F4FE19A8832784FDF2
:10171000C183232CF4FC832744FEE1072322F4FE3B
:10172000832744FE9843832784FDF98F89C7854723
:101730002326F4FE19A0232604FE8327C4FE3E853B
:10174000325445618280011122CE00102326A4FE6E
:101750008327C4FEFD8B0547B316F70037E700E08B
:101760008327C4FE9583938707048A07BA9794C397
:101770000100724405618280011122CE00102326EF
:10178000A4FE8327C4FEFD8B0547B316F70037E799
:1017900000E08327C4FE9583938707068A07BA97DC
:1017A00094C30100724405618280011122CE0010B1
:1017B0002326A4FEAE87A305F4FE37E700E08327C7
:1017C000C4FEBA970347B4FE2380E7400100724489
:1017D00005618280011122CE00102326A4FE03277A
:1017E000C4FE23ACE18001007244056182807971FE
:1017F00006D622D40018232EA4FCA30704FE83A738
:10180000818199EF8327C4FD9C233E878327C4FDF4
:10181000BC23920793F7F70FBE853A85793771AAF3
:1018200003A781818547631AF7048327C4FD983392
:1018300085476316F7028327C4FD9C233E878327D1
:10184000C4FDBC239207E207E18793E707F8E207AC
:10185000E18793F7F70FBE853A85813FB9AA8327C1
:10186000C4FD9C233E878327C4FDBC23920793F7C6
:10187000F70FBE853A85153F89A203A78181894765
:101880006314F7088327C4FD9833854763EBE702A9
:101890008327C4FDB8238327C4FD9C338A0793F7AD
:1018A000F70FBA97A307F4FE8327C4FD9C233E8756
:1018B0008347F4FE920793F7F70FBE853A85F53517
:1018C000EDA88327C4FDB8238327C4FD9C339387E9
:1018D000E70393F7F70F8A0793F7F70FBA97A30772
:1018E000F4FE8327C4FD9C233E878347F4FE9207C2
:1018F000E207E18793E707F8E207E18793F7F70F3D
:10190000BE853A855D3555A803A781818D4763144F
:10191000F7088327C4FD98338D4763EBE7028327DD
:10192000C4FDB8238327C4FD9C33860793F7F70FC4
:10193000BA97A307F4FE8327C4FD9C233E87834701
:10194000F4FE920793F7F70FBE853A85B93DB5A02F
:101950008327C4FDB8238327C4FD9C339387C7071F
:1019600093F7F70F860793F7F70FBA97A307F4FEDD
:101970008327C4FD9C233E878347F4FE9207E2073A
:10198000E18793E707F8E207E18793F7F70FBE8552
:101990003A85213D1DA003A781819147631FF70070
:1019A0008327C4FD9C233E878327C4FD9C33920775
:1019B00093F7F70FBE853A85CD3B8327C4FDDC4303
:1019C00099C78327C4FD9C233E85B53B31A083275F
:1019D000C4FD9C233E854D330100B2502254456125
:1019E0008280797122D60018232EA4FC232604FEBF
:1019F000B7170240DC432326F4FE0327C4FED17749
:101A0000FD17F98F2326F4FE0327C4FE8327C4FDA8
:101A1000D98F2326F4FEB71702400327C4FED8C38C
:101A20000100325445618280797122D60018232E3C
:101A3000A4FC232404FE232604FE232204FE2320E8
:101A400004FEB7170240DC43B18B2324F4FE0327C6
:101A500084FE91476303F702032784FEA1476306D0
:101A6000F702832784FE639607108327C4FD371788
:101A70007A001307072098C329A28327C4FD37578C
:101A8000E8011307078098C3EDA8B7170240D843B1
:101A9000B7073C00F98F2326F4FEB7170240D8435E
:101AA000C167F98F2322F4FE8327C4FEC983890707
:101AB0002326F4FE0327C4FEC5476315F700C94774
:101AC0002326F4FE832744FEA1E3B7470240938711
:101AD00007809C43C18B89CF0327C4FEB7177A00C8
:101AE000938707203307F7028327C4FD98C351A8C3
:101AF0000327C4FEB7173D00938707903307F7020B
:101B00008327C4FD98C3B5A8B7170240D843B707C9
:101B1000C0007D8FB707C000631EF7000327C4FE17
:101B2000B727F400938707403307F7028327C4FDE4
:101B300098C381A8B7170240D843B7070200F98FAE
:101B400089CF0327C4FEB7173D009387079033075B
:101B5000F7028327C4FD98C32DA00327C4FEB7173F
:101B60007A00938707203307F7028327C4FD98C3C1
:101B700009A88327C4FD37177A001307072098C3E5
:101B80000100B7170240DC4393F7070F2324F4FE4C
:101B9000832784FE91832324F4FEB7070020138754
:101BA0000700832784FEBA979C2393F7F70F23201F
:101BB000F4FE8327C4FD9843832704FE3357F700C0
:101BC0008327C4FDD8C3B7170240DC4393F70770DF
:101BD0002324F4FE832784FEA1832324F4FEB70785
:101BE000002013870700832784FEBA979C2393F76E
:101BF000F70F2320F4FE8327C4FDD843832704FE78
:101C00003357F7008327C4FD98C7B7170240D8435E
:101C1000916793870780F98F2324F4FE832784FE3E
:101C2000AD832324F4FEB707002013870700832722
:101C300084FEBA979C2393F7F70F2320F4FE8327A3
:101C4000C4FDD843832704FE3357F7008327C4FD20
:101C5000D8C7B7170240D843B167F98F2324F4FEE1
:101C6000832784FEB9832324F4FEB707002013875B
:101C7000471E832784FEBA979C2393F7F70F2320F0
:101C8000F4FE8327C4FDD847832704FE3357F702A9
:101C90008327C4FD98CB0100325445618280011135
:101CA00022CE00102326A4FE2324B4FE832784FE24
:101CB00099CBB7170240D44BB71702400327C4FE95
:101CC000558FD8CB21A8B7170240D44B8327C4FE29
:101CD00013C7F7FFB7170240758FD8CB01007244C6
:101CE00005618280011122CE00102326A4FE232448
:101CF000B4FE832784FE99CBB7170240944FB717E1
:101D000002400327C4FE558F98CF21A8B717024081
:101D1000944F8327C4FE13C7F7FFB7170240758F90
:101D200098CF0100724405618280011122CE00101B
:101D30002326A4FE2324B4FE832784FE99CBB71761
:101D40000240D44FB71702400327C4FE558FD8CFA7
:101D500021A8B7170240D44F8327C4FE13C7F7FF4B
:101D6000B7170240758FD8CF010072440561828099
:101D7000011122CE00102326A4FE2324B4FE8327C3
:101D800084FE99CBB7170240D447B7170240032708
:101D9000C4FE558FD8C721A8B7170240D447832760
:101DA000C4FE13C7F7FFB7170240758FD8C70100ED
:101DB000724405618280797122D60018232EA4FC1A
:101DC000232CB4FC231704FE8327C4FD9E23231772
:101DD000F4FE0327C4FDB7370140938707C06300B3
:101DE000F7040327C4FDB7070040630AF70203277F
:101DF000C4FDB7070040938707406302F70203273B
:101E0000C4FDB717004093870780630AF7000327D4
:101E1000C4FDB7170040938707C06310F7028357CC
:101E2000E4FE93F7F7F82317F4FE832784FDBA2323
:101E30008357E4FED98F2317F4FE8357E4FE93F70C
:101E4000F7CF2317F4FE832784FDFA238357E4FE9C
:101E5000D98F2317F4FE8327C4FD0357E4FE9AA30A
:101E6000832784FDDA238327C4FDDAB7832784FD23
:101E70009A238327C4FD9AB70327C4FDB7370140CF
:101E8000938707C0631BF700832784FD9C27139764
:101E9000070141838327C4FD9ABB8327C4FD0547FF
:101EA000DAAB0100325445618280797122D6001884
:101EB000232EA4FC232CB4FC231504FE231704FEBC
:101EC000231604FE8327C4FD9E33C207C183F99BFA
:101ED0001397070141838327C4FD9AB38327C4FD69
:101EE0009E332317F4FE8327C4FDDE232316F4FE5E
:101EF0008327C4FD9E2F2315F4FE8357A4FE93F77A
:101F0000F7F82315F4FE8357A4FEF19B2315F4FE86
:101F1000832784FD9A238357A4FED98F2315F4FECB
:101F20008357E4FEF59B2317F4FE832784FD9A274D
:101F30008357E4FED98F2317F4FE832784FDBA2349
:101F40008357E4FED98F2317F4FE0327C4FDB73768
:101F50000140938707C06318F7068357E4FEDD9BB3
:101F60002317F4FE832784FDBA278357E4FED98F15
:101F70002317F4FE8357E4FEED9B2317F4FE83271B
:101F800084FDDA238357E4FED98F2317F4FE8357A9
:101F9000C4FE93F7F7EF2316F4FE8357C4FE93F7BE
:101FA000F7DF2316F4FE832784FDDA278357C4FE68
:101FB000D98F2316F4FE832784FDFA278357C4FEA6
:101FC000D98F2316F4FE8327C4FD0357C4FEDAA37A
:101FD0008327C4FD0357A4FE9AAF832784FDFA2309
:101FE0008327C4FDDABB8327C4FD0357E4FE9AB3FD
:101FF0000100325445618280797122D60018232E67
:10200000A4FC232CB4FC231504FE231704FE231682
:1020100004FE8327C4FD9E33C207C183BD9B139773
:10202000070141838327C4FD9AB38327C4FD9E33F0
:102030002317F4FE8327C4FDDE232316F4FE832733
:10204000C4FD9E2F2315F4FE0357A4FEE577FD176C
:10205000F98F2315F4FE8357A4FE93F7F7CF2315CA
:10206000F4FE832784FD9E23A20713970701418373
:102070008357A4FED98F2315F4FE8357E4FE93F70C
:10208000F7FD2317F4FE832784FD9E2792071397FD
:10209000070141838357E4FED98F2317F4FE83277A
:1020A00084FDBE2392071397070141838357E4FE03
:1020B000D98F2317F4FE0327C4FDB7370140938758
:1020C00007C0631CF7088357E4FE93F7F7F723175D
:1020D000F4FE832784FDBE279207139707014183EF
:1020E0008357E4FED98F2317F4FE8357E4FE93F75A
:1020F000F7FB2317F4FE832784FDDE239207139753
:10210000070141838357E4FED98F2317F4FE8357D9
:10211000C4FE93F7F7BF2316F4FE0357C4FEFD7702
:102120009387F77FF98F2316F4FE832784FDDE273C
:102130008A071397070141838357C4FED98F23165B
:10214000F4FE832784FDFE278A0713970701418346
:102150008357C4FED98F2316F4FE8327C4FD03578B
:10216000C4FEDAA38327C4FD0357A4FE9AAF8327D6
:1021700084FDFA238327C4FD9ABF8327C4FD035738
:10218000E4FE9AB30100325445618280797122D60F
:102190000018232EA4FC232CB4FC231504FE2317C3
:1021A00004FE231604FE8327C4FD9E33C207C183A9
:1021B00093F7F7EF1397070141838327C4FD9AB381
:1021C0008327C4FD9E332317F4FE8327C4FDDE233B
:1021D0002316F4FE8327C4FDDE2F2315F4FE835758
:1021E000A4FE93F7F7F82315F4FE8357A4FEF19BA2
:1021F0002315F4FE832784FD9A238357A4FED98FE9
:102200002315F4FE8357E4FE93F7F7DF2317F4FE5C
:10221000832784FD9E27A2071397070141838357D5
:10222000E4FED98F2317F4FE832784FDBE23A20783
:102230001397070141838357E4FED98F2317F4FED8
:102240000327C4FDB7370140938707C0631EF70813
:102250000357E4FEFD779387F77FF98F2317F4FE8A
:10226000832784FDBE27A207139707014183835765
:10227000E4FED98F2317F4FE8357E4FE93F7F7BFEC
:102280002317F4FE832784FDDE23A207139707019B
:1022900041838357E4FED98F2317F4FE0357C4FE0E
:1022A000FD77FD17F98F2316F4FE0357C4FEF97767
:1022B000FD17F98F2316F4FE832784FDDE2792078E
:1022C0001397070141838357C4FED98F2316F4FE69
:1022D000832784FDFE2792071397070141838357C5
:1022E000C4FED98F2316F4FE8327C4FD0357C4FE12
:1022F000DAA38327C4FD0357A4FEDAAF832784FD46
:10230000FA238327C4FDDABF8327C4FD0357E4FE05
:102310009AB30100325445618280797122D6001847
:10232000232EA4FC232CB4FC231604FE231504FE48
:10233000231704FE8327C4FD9E33139707014183AF
:10234000FD77FD17F98F1397070141838327C4FD9C
:102350009AB38327C4FD9E332315F4FE8327C4FD5F
:10236000DE232317F4FE8327C4FDDE2F2316F4FE9D
:102370000357C4FEE577FD17F98F2316F4FE835744
:10238000C4FE93F7F7CF2316F4FE832784FD9E2324
:10239000A2071397070141838357C4FED98F2316E1
:1023A000F4FE0357A4FEF977FD17F98F2315F4FE09
:1023B000832784FD9E27B207139707014183835724
:1023C000A4FED98F2315F4FE832784FDBE23B20714
:1023D0001397070141838357A4FED98F2315F4FE79
:1023E0000327C4FDB7370140938707C06315F70281
:1023F0000357E4FEF177FD17F98F2317F4FE8327C7
:1024000084FDDE279A071397070141838357E4FE73
:10241000D98F2317F4FE8327C4FD0357E4FEDAA304
:102420008327C4FD0357C4FEDAAF832784FDFA2354
:102430008327C4FD2390E7048327C4FD0357A4FE2C
:102440009AB30100325445618280011122CE0010FE
:102450002326A4FE2324B4FE832784FE99CF83275A
:10246000C4FE9E23C207C18393E717001397070199
:1024700041838327C4FE9AA329A88327C4FE9E23F1
:10248000C207C183F99B1397070141838327C4FEC9
:102490009AA30100724405618280011122CE0010CE
:1024A0002326A4FE2324B4FE832784FE95C383271A
:1024B000C4FE83D74704139707014183E177D98F7F
:1024C0001397070141838327C4FE2392E70415A0D5
:1024D0008327C4FE83D74704139707014183A1676D
:1024E000FD17F98F1397070141838327C4FE2392B9
:1024F000E7040100724405618280011122CE0010C0
:102500002326A4FEAE872322C4FE2315F4FE8327D0
:1025100044FE8DC38327C4FEDE2713970701418342
:102520008357A4FED98F1397070141838327C4FEE5
:10253000DAA725A08327C4FEDE271397070141836E
:102540008357A4FE93C7F7FFC207C183F98F139780
:10255000070141838327C4FEDAA7010072440561A5
:102560008280011122CE00102326A4FE2324B4FE73
:10257000832784FE99CF8327C4FE9E23C207C1838D
:1025800093E707081397070141838327C4FE9AA3A3
:1025900031A88327C4FE9E23C207C18393F7F7F7B0
:1025A0001397070141838327C4FE9AA30100724455
:1025B00005618280797122D60018232EA4FCAE8793
:1025C000231DF4FC231704FE8327C4FD9E2F23172D
:1025D000F4FE8357E4FEDD9B2317F4FE0357E4FE6D
:1025E0008357A4FDD98F2317F4FE8327C4FD035717
:1025F000E4FE9AAF0100325445618280797122D69F
:102600000018232EA4FCAE87231DF4FC231704FE20
:102610008327C4FD9E2F2317F4FE0357E4FEFD77A6
:102620009387F77FF98F2317F4FE8357A4FDA20742
:102630001397070141838357E4FED98F2317F4FED4
:102640008327C4FD0357E4FE9AAF0100325445616D
:102650008280797122D60018232EA4FCAE87231D18
:10266000F4FC231704FE8327C4FDDE2F2317F4FE9A
:102670008357E4FEDD9B2317F4FE0357E4FE8357E4
:10268000A4FDD98F2317F4FE8327C4FD0357E4FE6E
:10269000DAAF0100325445618280797122D6001888
:1026A000232EA4FCAE87231DF4FC231704FE8327EE
:1026B000C4FDDE2F2317F4FE0357E4FEFD77938756
:1026C000F77FF98F2317F4FE8357A4FDA207139712
:1026D000070141838357E4FED98F2317F4FE832734
:1026E000C4FD0357E4FEDAAF010032544561828035
:1026F000797122D60018232EA4FCAE87231DF4FC8A
:10270000232604FE231504FE231404FE8327C4FDA0
:102710009E2B1397070141838357A4FDF98F23153F
:10272000F4FE8327C4FDDE271397070141838357F7
:10273000A4FDF98F2314F4FE8357A4FE81CB8357A5
:1027400084FE89C785472326F4FE19A0232604FEAC
:102750008327C4FE3E85325445618280011122CE1A
:1027600000102326A4FEAE872315F4FE8357A4FE93
:1027700093C7F7FF1397070141838327C4FE9AABE2
:1027800001007244056182805D7186C6A2C4800822
:10279000232EA4FA232CB4FA232604FE232404FEB9
:1027A000232204FE232004FE232E04FC8327C4FBE3
:1027B000232EF4FC8327C4FB9E2BC207C183232650
:1027C000F4FE0327C4FEB567FD17F98F2326F4FE38
:1027D000832784FBFE233E878327C4FED98F2326CD
:1027E000F4FE8327C4FE1397070141838327C4FBAC
:1027F0009AAB8327C4FBDE27C207C1832326F4FEDE
:102800000327C4FEBD679387379FF98F2326F4FE05
:10281000832784FBDA23832784FB9E27D98F139792
:1028200007014183832784FBBE27D98FC207C18359
:102830003E878327C4FED98F2326F4FE8327C4FE58
:102840001397070141838327C4FBDAA78327C4FBBF
:10285000DE2BC207C1832326F4FE0327C4FEC16713
:102860009387F7CFF98F2326F4FE832784FBDE2797
:102870003E878327C4FED98F2326F4FE8327C4FE18
:102880001397070141838327C4FBDAAB930784FCCA
:102890003E85EFF06F990327C4FDB747014093874A
:1028A00007806317F700832744FD2324F4FE29A043
:1028B000832704FD2324F4FE8327C4FBDE27C207FD
:1028C000C183C207C18763D20702032784FEBA8788
:1028D0008607BA978E073E97832784FB9C4386071B
:1028E000B357F7022322F4FE05A0032784FEBA871C
:1028F0008607BA978E073E97832784FB9C438A07F7
:10290000B357F7022322F4FE032744FE9307400641
:10291000B357F70292072326F4FE8327C4FE13D78A
:10292000470093074006B307F702032744FEB307A7
:10293000F7402320F4FE8327C4FBDE27C207C183B0
:10294000C207C18763D20702832704FE8E0713875D
:10295000270393074006B357F7029D8B0327C4FE56
:10296000D98F2326F4FE05A0832704FE9207138740
:10297000270393074006B357F702BD8B0327C4FE16
:10298000D98F2326F4FE8327C4FE139707014183C2
:102990008327C4FB9AA70100B64026446161828068
:1029A000011122CE00102326A4FE2324B4FE832787
:1029B00084FE85C38327C4FEDE2713970701418366
:1029C0008967D98F1397070141838327C4FEDAA74C
:1029D00005A08327C4FEDE27139707014183F977FB
:1029E000FD17F98F1397070141838327C4FEDAA7E8
:1029F0000100724405618280797122D60018232E6D
:102A0000A4FCAE87232AC4FC231DF4FC232404FE6B
:102A1000232204FE232004FE232604FE8327C4FD74
:102A20002326F4FE8357A4FD93F7F70F958393F7BE
:102A3000F70F2324F4FE8357A4FDFD8B2322F4FE1D
:102A4000832744FE0547B317F7002320F4FE03272E
:102A500084FE85476318F7008327C4FEB107232649
:102A6000F4FE0DA0032784FE89476318F70083272F
:102A7000C4FEC1072326F4FE31A08327C4FED1077C
:102A80002326F4FE832744FD99CB8327C4FE944379
:102A90008327C4FE032704FE558F98C321A88327EC
:102AA000C4FE9443832704FE13C7F7FF8327C4FEA5
:102AB000758F98C30100325445618280011122CE86
:102AC00000102326A4FEAE872315F4FE8357A4FE30
:102AD00093F7F71F1397070141838327C4FEDAA3F7
:102AE0000100724405618280011122CE001023266C
:102AF000A4FE8327C4FEDE23C207C18393F7F71F1A
:102B0000C207C1833E85724405618280797122D6F5
:102B10000018232EA4FCAE87231DF4FC232204FE00
:102B2000232604FE232004FE232404FE8357A4FD51
:102B300093F7F70F958393F7F70F2320F4FE83574E
:102B4000A4FDFD8B2326F4FE8327C4FE0547B3179F
:102B5000F7002326F4FE032704FE8547631EF700D3
:102B60008327C4FDDE27C207C1833E878327C4FEB7
:102B7000F98F2326F4FE2DA8032704FE8947631E40
:102B8000F7008327C4FD9E2BC207C1833E8783279E
:102B9000C4FEF98F2326F4FE21A88327C4FDDE2B73
:102BA000C207C1833E878327C4FEF98F2326F4FE24
:102BB0008357A4FDA183C207C1832322F4FE832788
:102BC00044FE0547B317F7002322F4FE8327C4FD14
:102BD0009E23C207C1833E87832744FEF98F2322A9
:102BE000F4FE8327C4FE81CB832744FE89C7854733
:102BF0002324F4FE19A0232404FE832784FE3E85AB
:102C0000325445618280797122D60018232EA4FCAB
:102C1000AE87231DF4FC231704FE231604FE8357FE
:102C2000A4FDA1832317F4FE8357E4FE0547B317E1
:102C3000F7002316F4FE8357C4FE93C7F7FF1397DC
:102C4000070141838327C4FD9AA3010032544561E3
:102C50008280411122C60008B7F700E023A20700D6
:102C600001003244410173002030011106CE22CC14
:102C700000102326A4FE2324B4FE2322C4FE8327AF
:102C800044FE3E86832584FE138541A3EF10305D0C
:102C9000832744FE3E85F240624405618280011133
:102CA00022CE00102326A4FE03A781808327C4FE22
:102CB0003E979387C1CE636DF70003A7818083277A
:102CC000C4FE3E97B78700209387078063F4E70030
:102CD000FD5739A803A781808327C4FE3E9723A40C
:102CE000E18003A781808327C4FEB307F040BA9731
:102CF0003E85724405618280011106CE22CC4ACA0B
:102D00004EC80010232604FE49A80327C4FE060768
:102D100093870185BA979E23C207C1833E85EF4002
:102D20004028B16703A6877A83A6C77AEF3060068A
:102D3000AA872E883E85C285B16703A6077B83A636
:102D4000477BEF304060AA872E883E89C28983275F
:102D5000C4FE138701858A07BA979C473E85EF40DA
:102D6000003EAA872E883E86C2864A85CE85EF30F1
:102D7000805DAA872E883E85C285EF400047AA86DF
:102D80008327C4FE9107138701858A07BA9794C7E2
:102D90008327C4FE85072326F4FE0327C4FE8D4740
:102DA000E3D5E7F693870185984F9387018598D7F8
:102DB00093870185D84F93870185D8D7938701855D
:102DC00098539387018598DB93870185D853938720
:102DD0000185D8DB0100F24062445249C2490561D5
:102DE0008280597186D6A2D48018232404FE23261B
:102DF00004FE232404FC232604FC232804FC232AA9
:102E000004FC232C04FC232E04FC232004FE232298
:102E100004FE232E04FA232004FC232204FC23288E
:102E200004F8232A04F8232C04F8232E04F8232082
:102E300004FA232204FA232404FA232604FA23287A
:102E400004FA232A04FA232C04FA938701853167B4
:102E50000327877B98C79387018531670327C77B43
:102E6000D8C79387018531670327C77B98CB9387A2
:102E7000018531670327077CD8CB93870185238C95
:102E8000070285454145EFE0FFE585451305002034
:102E9000EFE05FE585450545EFE07FE085450545C9
:102EA000EFE05FE4BD47231EF4FA232204FC9307FE
:102EB000C4FBBE8537150140EFD01FF3B7070240B2
:102EC00013858700EFD0FFC3B72701409387C7441E
:102ED0002328F4F893870185232AF4F8232C04F897
:102EE0009147232EF4F8232004FA930700082322A5
:102EF000F4FA930700102324F4FA930700402326E2
:102F0000F4FA232804FA232A04FA232C04FA930758
:102F100004F9BE85B707024013858700EFD0FFD3C1
:102F2000ED472304F4FE8547A304F4FE230504FEC5
:102F300085472326F4FE930784FE3E85EFE03F8B12
:102F400005468945B707024013858700EFD07FDF2C
:102F50008545B707024013858700EFD09FDAB72772
:102F6000014013850740EFD06FD9232404FC854727
:102F70002326F4FC85472328F4FCB7070E00232AF8
:102F8000F4FC232C04FC9147230EF4FC930784FCEF
:102F9000BE85B727014013850740EFD02FDC316590
:102FA000EFE03FA49D460546A945B727014013859C
:102FB0000740EFD07F869D460946AD45B7270140C3
:102FC00013850740EFD05F859D460D46B145B72775
:102FD000014013850740EFD03F849D461146B5451B
:102FE000B727014013850740EFD01F838545B727DA
:102FF000014013850740EFD04FEA8545B7270140D0
:1030000013850740EFD08FE5B727014013850740B0
:10301000EFD00FF20100B727014013850740EFD032
:103020004FF3AA87EDFBB727014013850740EFD088
:103030004FF50100B727014013850740EFD08FF609
:10304000AA87EDFB930720022304F4FE8547A3041F
:10305000F4FE230504FE85472326F4FE930784FE31
:103060003E85EFE0CFF8054693050022B7270140E3
:1030700013850740EFD04FE68545B72701401385FC
:103080000740EFD02FF50100B650265465618280CD
:10309000797106D622D40018232EA4FCA30704FEBF
:1030A00083A7C1810327C4FD63F5E70283A7C1811C
:1030B0000327C4FD1D8FB7470F009387F72363FFD6
:1030C000E7028547A307F4FE0327C4FD23AEE18092
:1030D00035A083A7C1810327C4FDB307F740138739
:1030E000F7FFB7470F009387F72363F9E70085479A
:1030F000A307F4FE0327C4FD23AEE1808347F4FE5B
:10310000A9C79387018583C78703A1E3B707024057
:10311000A1071147D8C38545B7070240138587002B
:10312000EFD03FBE8545B727014013850740EFD05C
:10313000EFD28545B727014013850740EFD08FE9CF
:10314000938701850547238CE7020100B250225482
:1031500045618280411122C6000893050022B727ED
:10316000014013850740EFD0BF8FAA8789CB930515
:103170000022B727014013850740EFD01F950100BB
:103180003244410173002030411122C60008094534
:10319000EFD0DFBFAA879DC78145B72701401385C0
:1031A0000740EFD02FE38145B72701401385074043
:1031B000EFD0CFCA91360945EFD05FC19387018523
:1031C000238C070201003244410173002030411179
:1031D00006C622C40008E1679388076A054893077A
:1031E000000437170140130707C09306000837167D
:1031F0000140130606C0B75500409385054013856E
:10320000C1883528E1679388076A09489307004019
:1032100037170140130707C0856693860680371667
:103220000140130606C0B7650040938505801385ED
:10323000418A31200100B2402244410182805D7107
:1032400086C6A2C480082326A4FC2324B4FC23221F
:10325000C4FC2320D4FC232EE4FA232CF4FAC287E6
:10326000232814FBA30BF4FA232004FE232204FEDC
:10327000232404FE232804FC232A04FC232C04FC1E
:10328000232E04FCB70720002326F4FE8327C4FC6A
:10329000032784FC98C38327C4FC032744FCD8C3BA
:1032A0008327C4FC032704FCD8C78327C4FC032757
:1032B000C4FB98C78327C4FC032784FB98CB8327D0
:1032C000C4FC034774FBF8AB85450545EFE09FA1BF
:1032D0008327C4FC9843B757004093870740631780
:1032E000F700B70720002326F4FE31A88327C4FC8B
:1032F0009843B7670040938707806316F700B707C6
:1033000040002326F4FE85450325C4FEEFE0FFA11F
:103310008327C4FCD843B7170140938707806316FF
:10332000F70091472326F4FEA5A08327C4FCD843C9
:10333000B7170140938707C06316F700A1472326FC
:10334000F4FEB9A08327C4FCD843B7170140631625
:10335000F700C1472326F4FE25A88327C4FCD843E1
:10336000B7170140938707406317F70093070002E0
:103370002326F4FE31A88327C4FCD843B727014095
:10338000938707806316F700930700042326F4FE53
:1033900085450325C4FEEFE0FF948327C4FCDC478A
:1033A000C207C1832310F4FEF1472324F4FE8D47A6
:1033B0002322F4FE8327C4FCDC43130704FEBA85F2
:1033C0003E85EFD07FA28327C4FC9847B717014002
:1033D000938707806316F70091472326F4FEA5A084
:1033E0008327C4FC9847B7170140938707C063162B
:1033F000F700A1472326F4FEB9A08327C4FC984711
:10340000B71701406316F700C1472326F4FE25A82D
:103410008327C4FC9847B717014093870740631779
:10342000F700930700022326F4FE31A88327C4FC8B
:103430009847B7270140938707806316F7009307E3
:1034400000042326F4FE85450325C4FEEFE09F8992
:103450008327C4FC9C4BC207C1832310F4FEF147B1
:103460002324F4FE8D472322F4FE8327C4FC9C47CB
:10347000130704FEBA853E85EFD01F97832704FB10
:103480002328F4FC231A04FC9167231BF4FC930704
:10349000000A231CF4FC93070040231DF4FC9167F1
:1034A000231EF4FC8327C4FC9C43130704FDBA8548
:1034B0003E85EFD03FD98327C4FC9C4385453E859C
:1034C000EFD0FFF90100B64026446161828031717E
:1034D00006DF22DD26DB80012326A4F4AE8723222B
:1034E000D4F42315F4F4B2872314F4F4BA87231127
:1034F000F4F4A30704FE01008327C4F49C43B7053A
:1035000002003E85EFE0AF9BAA87FDF78327C4F456
:103510009C4385453E85EFD09FF901008327C4F485
:103520009843B7070300938517003A85EFE0EF90C3
:10353000AA87EDD78327C4F49C430357A4F41377D9
:10354000F70F0146BA853E85EFE04F8A01008327D9
:10355000C4F49843B7070700938527083A85EFE03E
:10356000CF8DAA87EDD78327C4F4F82B854763193D
:10357000F702835784F493F7F70F230EF4F49307BD
:10358000C4F58507035724F43A86832544F43E8521
:10359000EF3070648347F4FE8507A307F4FE81A033
:1035A000835784F4A183C207C18393F7F70F230ED7
:1035B000F4F4835784F493F7F70FA30EF4F493070E
:1035C000C4F58907035724F43A86832544F43E85DD
:1035D000EF3070608347F4FE8907A307F4FE2324CD
:1035E00004FE89A08327C4F49843832784FE9306AE
:1035F00004FFB69783C7C7F6BE853A85EFD09FFA1A
:1036000001008327C4F49843B70707009385470850
:103610003A85EFE08F82AA87EDD7832784FE85075E
:103620002324F4FE8347F4FE032784FEE34CF7FAD9
:103630008327C4F49C4385453E85EFD05FE70100B6
:103640008327C4F49843B7070300938517003A858E
:10365000EFD0BFFEAA87EDD78327C4F49C4303575E
:10366000A4F41377F70F0546BA853E85EFD01FF80F
:1036700001008327C4F49843B7070300938527000C
:103680003A85EFD09FFBAA87EDD701A88327C4F422
:103690009C4385453E85EFD0DFEB8327C4F49843F8
:1036A000B7070010938507043A85EFE04F81AA879A
:1036B000F1DF231304FE91A08327C4F49C438354B9
:1036C00064FE3E85EFD09FF0AA873E87930704FFF4
:1036D000A697238AE7F601008327C4F49843B70727
:1036E0000300938507043A85EFD03FF5AA87EDD70D
:1036F000835764FE85072313F4FE035764FE835744
:1037000024F4FD17E34AF7FA8327C4F49C43835457
:1037100064FE3E85EFD09FEBAA873E87930704FFA8
:10372000A697238AE7F68327C4F49C4385453E8504
:10373000EFD01FDD035764FE930744F63A86BE853B
:10374000032544F4EF303049835764FE3E85FA5038
:103750006A54DA5429618280717106D722D5001922
:10376000232EA4F4AE87232AD4F4231DF4F4B287C5
:10377000231CF4F4BA872319F4F4835724F5A30720
:10378000F4FE01008327C4F59C43B70502003E8583
:10379000EFD0FFF2AA87FDF78327C4F59C43854548
:1037A0003E85EFD0DFD001008327C4F59843B707EB
:1037B0000300938517003A85EFD03FE8AA87EDD73D
:1037C0008327C4F59C430357A4F51377F70F0146ED
:1037D000BA853E85EFD09FE101008327C4F5984369
:1037E000B7070700938527083A85EFD01FE5AA871A
:1037F000EDD78327C4F5F82B85476319F702835764
:1038000084F593F7F70F2306F4F69307C4F68507BC
:10381000035724F53A86832544F53E85EF30B03BC7
:103820008347F4FE8507A307F4FE81A0835784F540
:10383000A183C207C18393F7F70F2306F4F68357DA
:1038400084F593F7F70FA306F4F69307C4F68907F8
:10385000035724F53A86832544F53E85EF30B0378B
:103860008347F4FE8907A307F4FE231604FE89A00C
:103870008327C4F598438357C4FE930604FFB69785
:1038800083C7C7F7BE853A85EFD0DFD10100832714
:10389000C4F59843B7070700938547083A85EFD0EA
:1038A000DFD9AA87EDD78357C4FE85072316F4FE18
:1038B0008347F4FEC207C1830357C4FEE36AF7FAE5
:1038C0008327C4F59C4385453E85EFD07FC383574E
:1038D000C4FE3E85BA502A544D618280411106C60D
:1038E00022C4000881461146B7170140938507405E
:1038F0001385C18BBD2081462146B71701409385B2
:1039000007C01385018FB12881464146B717014092
:10391000938507C013854192A920814613060002B2
:10392000B7170140938507C0138581951D280100B5
:10393000B240224441018280411106C622C40008DF
:103940001385C18BB1221385018F99221385419272
:103950008122138581952D2A0100B2402244410124
:103960008280797106D622D40018232EA4FC232C41
:10397000B4FC232AC4FCB687A309F4FC8327C4FD46
:10398000638307108327C4FD032784FD98C383271F
:10399000C4FD032744FDD8C38327C4FD034734FD7A
:1039A000D8AF8327C4FD514798C78327C4FD23AAF6
:1039B00007008327C4FD23A807008327C4FD23AC89
:1039C0000700232004FE232204FE232404FE832771
:1039D000C4FD9843B7170140938707806316F7002B
:1039E00091472326F4FEA5A08327C4FD9843B7176B
:1039F0000140938707C06316F700A1472326F4FE12
:103A0000B9A08327C4FD9843B71701406316F70098
:103A1000C1472326F4FE25A88327C4FD9843B71782
:103A20000140938707406317F7009307000223269E
:103A3000F4FE31A88327C4FD9843B727014093873C
:103A400007806316F700930700042326F4FE8545DC
:103A50000325C4FEEFE00FA98327C4FDDC43C207A2
:103A6000C1832310F4FE91472324F4FE89472322C7
:103A7000F4FE8327C4FD9C43130704FEBA853E85EC
:103A8000EFD08FB611A00100B25022544561828060
:103A9000797106D622D40018232EA4FC8327C4FDF6
:103AA00098438327C4FDDC43C207C183BE853A85A2
:103AB000EFD0AFD5AA87B337F00093F7F70FA3077E
:103AC000F4FE8327C4FDDC2F89C70547638EE7001A
:103AD0003DA08347F4FE93B7170093F7F70F3E8797
:103AE0008327C4FD98CF21A88347F4FEB337F000A5
:103AF00093F7F70F3E878327C4FD98CF0100D92E97
:103B00002A878327C4FDDC471D8F8327C4FD944784
:103B10009307803EB387F6026362F70A652E2A8711
:103B20008327C4FDD8C78327C4FDDC4B95EF8327CB
:103B3000C4FD984F8327C4FDDC4B630BF706832736
:103B4000C4FD984B8327C4FDDC4B6313F706832722
:103B5000C4FD0547D8CB8327C4FDDC53B1CB8327F5
:103B6000C4FDDC538297A9A08327C4FD984F832707
:103B7000C4FDDC4B630EF7028327C4FD984B8327FB
:103B8000C4FDDC4B6316F7028327C4FD23AA07009C
:103B90008327C4FD9C5789C78327C4FD9C57829700
:103BA0008327C4FDDC5789C78327C4FDDC57829770
:103BB0008327C4FD984F8327C4FD98CB0100B250E2
:103BC000225445618280411106C622C40008014783
:103BD00093060008B717014013860780B1679385E5
:103BE000477C1385C19861280147C14637160140BB
:103BF000B1679385877C1385419A512001479306CD
:103C0000000237160140B1679385077D1385C19B7C
:103C1000BD20014793060002B717014013860780B5
:103C2000B1679385877D1385419D91280147A166E2
:103C3000B717014013860780B1679385077E138508
:103C4000C19E35280147A146B7170140138607409A
:103C5000B1679385877E138541A015200147C14632
:103C6000B717014013860780B1679385077F1385D7
:103C7000C1A131200100B24022444101828039714A
:103C800006DE22DC80002326A4FC2324B4FC2322AD
:103C9000C4FCB6872311F4FCBA87A300F4FC232EDE
:103CA00004FC232004FE232204FE032744FCB71750
:103CB0000140938707806316F70091472326F4FE9F
:103CC00085A0032744FCB7170140938707C06316FC
:103CD000F700A1472326F4FEA1A0032744FCB71751
:103CE00001406316F700C1472326F4FE15A80327F9
:103CF00044FCB7170140938707406317F700930709
:103D000000022326F4FE29A8032744FCB72701401C
:103D1000938707806316F700930700042326F4FEB9
:103D200085450325C4FEEFD0FFFB835724FC231EEB
:103D3000F4FCC1472322F4FE89472320F4FE9307B5
:103D4000C4FDBE85032544FCEFD00F8A8327C4FC45
:103D500023AA07008327C4FC032784FC98C3832776
:103D6000C4FC035724FCDAA78327C4FC032744FCC4
:103D700098C78327C4FC238707008327C4FC130745
:103D8000803E98CB834714FC8DC38327C4FC98479F
:103D90008327C4FCDE270146BE853A85EFD08FAA73
:103DA0008327C4FC0547F8A705A08327C4FC9847D0
:103DB0008327C4FCDE270546BE853A85EFD08FA851
:103DC0008327C4FC2387070083A701829DCF83A795
:103DD00001822324F4FE31A0832784FEDC4B2324BC
:103DE000F4FE832784FEDC4BE5FB832784FE032758
:103DF000C4FCD8CB832784FEDE23850713970701F5
:103E000041838327C4FCDAA329A00327C4FC23A091
:103E1000E1820100F250625421618280797106D6FC
:103E200022D40018AA87231FF4FC83A70182B5CBF4
:103E300083A701822326F4FE8DA08327C4FEDE2300
:103E40000357E4FD6316F7048327C4FEFC278DE3C4
:103E50008327C4FE98478327C4FEDE270146BE851C
:103E60003A85EFD02F9E8327C4FE0547F8A715A8F3
:103E70008327C4FE98478327C4FEDE270546BE85F8
:103E80003A85EFD02F9C8327C4FE2387070011A813
:103E90008327C4FEDC4B2326F4FE8327C4FED1FF18
:103EA00009A00100B250225445618280411106C62A
:103EB00022C400080520AA873E85B2402244410161
:103EC0008280411122C6000883A741823E85324488
:103ED00041018280411122C60008B7370140938713
:103EE00007C0DE33C207C1833E8783A78182BA97AA
:103EF0003E85324441018280797106D622D4001871
:103F0000232EA4FC7D3F2326A4FE653F2A8783271A
:103F1000C4FEB307F7400327C4FD63F3E700F5B71A
:103F200001000100B250225445618280411122C635
:103F300000088545B7370140138507C0EFE04FFB08
:103F4000AA8785C783A781821387873E23A4E1823E
:103F500083A741821387170023A2E1828545B737E3
:103F60000140138507C0EFE06FFF010032444101BB
:103F700073002030411122C600088545B717004064
:103F8000138507C0EFE0CFF6AA8781CB8545B71729
:103F90000040138507C0EFE06FFC0100324441018F
:103FA00073002030411106C622C400081D203120B4
:103FB0000100B240224441018280411106C622C460
:103FC0000008D1280D2CE9260100B240224441010D
:103FD0008280797106D622D40018232204FE23247D
:103FE00004FE231604FE232E04FC232004FE854534
:103FF000856713850780EFD0FFCEB707002003A7A2
:10400000071EB7470F0093870724B357F702C2076D
:10401000C183FD17C207C1832312F4FE9307703ECC
:104020002314F4FE231504FE231304FE930744FE19
:10403000BE85B7370140138507C0EFD0DFD7854570
:10404000B7370140138507C0EFE0AFD1054685457E
:10405000B7370140138507C0EFE02FCA8545B73752
:104060000140138507C0EFE04FBE93079002230E77
:10407000F4FCA30E04FC8547230FF4FC85472320A2
:10408000F4FE9307C4FD3E85EFD06FF60100B250F9
:10409000225445618280397106DE22DC80002322B1
:1040A00004FE232404FE232604FE232A04FC232CDE
:1040B00004FC232E04FC232004FE232404FC2326DA
:1040C00004FC231804FC85451145EFD0BFC185458C
:1040D0000545EFD09FC5BD472312F4FEE1472326D7
:1040E000F4FE8D472324F4FE930744FEBE85B717E4
:1040F000014013850780EFC03FCFB707002003A71B
:10410000071EB7470F0093870724B357F702C2076C
:10411000C183FD17C207C1832314F4FC95679387FD
:10412000F7E12316F4FC231704FC231504FC930782
:1041300084FCBE8537050040EFD0FFC7930700061B
:10414000231AF4FC8547231BF4FC231E04FC93076D
:10415000803E231DF4FC930744FDBE8537050040D7
:10416000EFD0BFD49307803E231DF4FC930744FD9A
:10417000BE8537050040EFD03FE89307803E231D02
:10418000F4FC930744FDBE8537050040EFE00F8047
:104190009307803E231DF4FC930744FDBE8537053D
:1041A0000040EFE08F97A14537050040EFE08FC05A
:1041B000A14537050040EFE06FC4A1453705004039
:1041C000EFE02FC9A14537050040EFE00FCD854551
:1041D00037050040EFE0EFB8854537050040EFE0D8
:1041E000CFAB854537050040EFE02FA60100F25028
:1041F000625421618280397106DE22DC8000232234
:1042000004FE232404FE232604FE232A04FC232C7C
:1042100004FC232E04FC232004FE232404FC232678
:1042200004FC231804FC85454545EFD0BFAB85450C
:104230000945EFD09FAF8545B7171A00138507C012
:10424000EFC0DFE39307003C2312F4FEE14723268F
:10425000F4FE8D472324F4FE930744FEBE853715F4
:104260000140EFC07FB8B707002003A7071EB7477C
:104270000F0093870724B357F702C207C183FD17C6
:10428000C207C1832314F4FC9307703E2316F4FC89
:10429000231704FC231504FC930784FCBE85B70791
:1042A000004013850740EFD01FB193070006231A83
:1042B000F4FC8547231BF4FC231E04FC93074006F3
:1042C000231DF4FC930744FDBE85B707004013850A
:1042D0000740EFD09FBD93074006231DF4FC9307D2
:1042E00044FDBE85B707004013850740EFD0DFD0FF
:1042F00093074006231DF4FC930744FDBE85B707D2
:10430000004013850740EFD07FE893074006231D48
:10431000F4FC930744FDBE85B707004013850740B2
:10432000EFD0BFFFA145B707004013850740EFE07E
:104330006FA8A145B707004013850740EFE00FAC19
:10434000A145B707004013850740EFE08FB0A145B6
:10435000B707004013850740EFE02FB48545B70746
:10436000004013850740EFE0CF9F8545B707004029
:1043700013850740EFE06F928545B707004013852E
:104380000740EFE08F8C0100F2506254216182807F
:10439000397106DE22DC8000232204FE232404FE81
:1043A000232604FE232A04FC232C04FC232E04FCD5
:1043B000232004FE232404FC232604FC231804FCED
:1043C00085452145EFD01F9285451145EFD0FF95DA
:1043D000930700302312F4FEE1472326F4FE8D47B5
:1043E0002324F4FE930744FEBE85B71701401385CE
:1043F00007C0EFC07F9FB707002003A7071EB7477E
:104400000F0093870724B357F702C207C183FD1734
:10441000C207C1832314F4FC95679387F7E1231641
:10442000F4FC231704FC231504FC930784FCBE85CD
:10443000B717004013850780EFD0FF97930700065A
:10444000231AF4FC8547231BF4FC231E04FC93076A
:10445000803E231DF4FC930744FDBE85B717004042
:1044600013850780EFD09FD29307803E231DF4FC75
:10447000930744FDBE85B717004013850780EFD032
:10448000DFE9A145B717004013850780EFE08F9261
:10449000A145B717004013850780EFE02F96A1458F
:1044A000B717004013850780EFE0AF9AA145B71713
:1044B000004013850780EFE04F9E8545B717004009
:1044C00013850780EFE0EF898545B7170040138516
:1044D0000780EFD09FFC8545B71700401385078004
:1044E000EFD0BFF60100F2506254216182807971F1
:1044F00006D622D40018930700083EC89307000888
:104500003EC602C402C202C0F16793880720014878
:1045100093070040371701401307078093060020D8
:104520003716014013060680B74501409385058084
:10453000138541A3B120930700083EC893070008E4
:104540003EC602C402C202C09567938807B0B7078F
:104550001400138807018567938707803717014088
:104560009306004037160140B755004093850580FB
:10457000138541B331200100B2502254456182803D
:104580001D7186CEA2CC8010232EA4FA232CB4FA5F
:10459000232AC4FA2328D4FA2326E4FA2324F4FA9B
:1045A000232204FB232014FB232E04FC232004FEDF
:1045B000232204FE232604FC232804FC232A04FCD3
:1045C000232C04FC232204FC232404FC91672326CF
:1045D000F4FE8327C4FB032784FB98C38327C4FB13
:1045E000032744FBD8C38327C4FB032704FBD8C796
:1045F0008327C4FB0327C4FA98C78327C4FB032778
:1046000084FA98CB8327C4FBDC4B99C78327C4FB70
:10461000DC4B3E85EF20905B8327C4FB9C4F99C702
:104620008327C4FB9C4F3E85EF20505A0848EF205B
:104630005059AA873E878327C4FBD8CB4844EF2034
:104640005058AA873E878327C4FB98CF8327C4FB93
:104650001848D8D78327C4FB584498DB5C4413D749
:1046600017008327C4FBD8DB8327C4FB9843B747D5
:10467000014093870780631BF70091672326F4FEB0
:1046800085450325C4FEEFD0EFE58DA88327C4FB45
:104690009843B747004093870740631CF700B7076C
:1046A00002002326F4FE85450325C4FEEFD0EFE784
:1046B000B1A08327C4FB9843B75700409387078076
:1046C000631CF700B70704002326F4FE8545032585
:1046D000C4FEEFD08FE51DA08327C4FB9843B757D6
:1046E0000040938707C0631BF700B7070800232625
:1046F000F4FE85450325C4FEEFD02FE3854505452F
:10470000EFD04FDE832744FA91C78545032544FA4D
:10471000EFC0DF968327C4FBD843B71701409387C8
:1047200007806316F70091472326F4FEA5A0832790
:10473000C4FBD843B7170140938707C06316F7003F
:10474000A1472326F4FEB9A08327C4FBD843B7179B
:1047500001406316F700C1472326F4FE25A88327EE
:10476000C4FBD843B7170140938707406317F7008E
:10477000930700022326F4FE31A88327C4FBD84305
:10478000B7270140938707806316F700930700045B
:104790002326F4FE85450325C4FEEFD0AFD483273E
:1047A000C4FBDC47C207C183231EF4FCE14723227C
:1047B000F4FE8D472320F4FE8327C4FBDC4313075C
:1047C000C4FDBA853E85EFC02FE28327C4FB98471E
:1047D000B7170140938707806316F7009147232698
:1047E000F4FEA5A08327C4FB9847B7170140938721
:1047F00007C06316F700A1472326F4FEB9A083275C
:10480000C4FB9847B71701406316F700C14723263A
:10481000F4FE25A88327C4FB9847B7170140938768
:1048200007406317F700930700022326F4FE31A820
:104830008327C4FB9847B7270140938707806316F7
:10484000F700930700042326F4FE85450325C4FEE4
:10485000EFD04FC98327C4FB9C4BC207C183231EE3
:10486000F4FC91472322F4FE8D472320F4FE832796
:10487000C4FB9C471307C4FDBA853E85EFC0CFD665
:10488000832704FA2326F4FC1E202318F4FC5E2060
:104890002319F4FC1E24231AF4FC231C04FCB14746
:1048A000231BF4FC8327C4FB9C431307C4FCBA8579
:1048B0003E85EFD07FED8327C4FB9C4305469305DF
:1048C00050523E85EFE04F938327C4FB9C4305463F
:1048D000930540423E85EFE02F928327C4FB9C4323
:1048E0000146930570723E85EFE00F9193075003E8
:1048F000A305F4FE8327C4FB9843B7470140938781
:1049000007806317F70093075003A305F4FE91A8EF
:104910008327C4FB9843B74700409387074063173A
:10492000F70093076003A305F4FE25A88327C4FBC3
:104930009843B7570040938707806317F7009307A2
:104940007003A305F4FE31A88327C4FB9843B7572F
:104950000040938707C06316F70093072004A30560
:10496000F4FE8347B4FE2302F4FC8547A302F4FC63
:1049700085472303F4FC85472324F4FC930744FC78
:104980003E85EFC0DFE68327C4FB9C4385453E851B
:10499000EFE00F810100F640664425618280797165
:1049A00022D60018232EA4FC232CB4FC232AC4FCFA
:1049B000232604FE8327C4FDDC57C1CF8327C4FD13
:1049C000D84F8327C4FD9C53B307F7402324F4FE3C
:1049D0008327C4FDBC5B032784FE63F4E7068327BB
:1049E000C4FD032784FEB8DBA9A88327C4FD985320
:1049F0008327C4FDDC4F630DF7048327C4FDD84B28
:104A00008327C4FD9C53138617008326C4FD90D2D0
:104A10003E97832684FD8327C4FEB697182398A368
:104A20008327C4FD98538327C4FDDC576366F700D2
:104A30008327C4FD23A007028327C4FE85072326FE
:104A4000F4FE0327C4FE832744FDE360F7FA11A0B8
:104A500001008327C4FE3E8532544561828079710E
:104A600006D622D40018232EA4FC232CB4FC232A1F
:104A7000C4FC832744FD2322F4FE8327C4FDFC43AA
:104A8000138717008327C4FDF8C38327C4FD9C5BED
:104A9000F5C3232604FEA9A0032784FD8327C4FEB3
:104AA0003E978327C4FD944F8327C4FDDC53938531
:104AB00017000326C4FD4CD2B697182398A383276A
:104AC000C4FDD8538327C4FD9C5B6366F70083272E
:104AD000C4FD23A207028327C4FE85072326F4FE14
:104AE0000327C4FE832744FDE368F7FA8327C4FD48
:104AF000D8538327C4FD9C57B307F7402324F4FE03
:104B0000832784FE63DA07008327C4FD985B83272D
:104B100084FEBA972324F4FE8327C4FDF85B832721
:104B200084FE6377F700032784FE8327C4FDF8DB48
:104B30008327C4FD98578327C4FDDC53630CF70219
:104B40008327C4FDBC5F91CF8327C4FDB85F832753
:104B5000C4FDFC5FC207C1830546BE853A85EFC030
:104B60006FCE8327C4FD9C430546930570723E8536
:104B7000EFD09FE8832744FE3E85B2502254456122
:104B80008280011106CE22CC00102326A4FE8327AA
:104B9000C4FE9C43930550523E85EFD03FF7AA8751
:104BA000A1CF8327C4FE9C433E85EFD0FFF3AA87A5
:104BB000BE858327C4FED84B8327C4FEDC4F1386F3
:104BC00017008326C4FED0CEBA9713F7F50F98A32B
:104BD0008327C4FE9C5F138717008327C4FE98DFDA
:104BE0008327C4FED84F8327C4FEDC576366F700D3
:104BF0008327C4FE23AE07008327C4FE9C4393058E
:104C000040423E85EFD09FF0AA8799CF8327C4FE0C
:104C10009C43930540423E85EFD0FFFE8327C4FEB0
:104C20009C433E85EFD05FEC8327C4FE9C439305F5
:104C300070723E85EFD09FEDAA87C9CF8327C4FE4F
:104C40009C43930570723E85EFD0FFFB8327C4FE23
:104C500098578327C4FEDC536315F7028327C4FEED
:104C60009C430146930570723E85EFD0FFD88327A1
:104C7000C4FE9C430546930560623E85EFD0DFD7B6
:104C800091A88327C4FE88438327C4FE984F8327B7
:104C9000C4FE9C57138617008326C4FE90D6BA978D
:104CA0009C23C207C183BE85EFD05FE18327C4FE8A
:104CB000DC5F138717008327C4FED8DF8327C4FE79
:104CC00098578327C4FE9C5B6366F7008327C4FE66
:104CD00023A407028327C4FE9C43930560623E859C
:104CE000EFD0DFE2AA87B9C38327C4FE9C439305B4
:104CF00060623E85EFD03FF18327C4FE9C430146AE
:104D0000930560623E85EFD03FCF8327C4FEBC5F32
:104D100091CF8327C4FEB85F8327C4FEFC5FC20720
:104D2000C1830146BE853A85EFC0CFB10100F24094
:104D3000624405618280411122C60008138541A3A7
:104D4000893501003244410173002030411122C6EF
:104D50000008138541AB3535010032444101730031
:104D60002030411122C60008138541B3193D0100CE
:104D70003244410173002030011122CE001023265D
:104D8000A4FE2324B4FEB2872313F4FE8327C4FEBB
:104D9000035764FEDAA38327C4FE032784FE98C367
:104DA0008327C4FE373700001307E74C98C78327D3
:104DB000C4FE3737000013078775D8C70100724457
:104DC00005618280797106D622D40018232EA4FCB6
:104DD000AE87232AC4FC3687A30DF4FCBA87231CB4
:104DE000F4FC231704FE8327C4FD03A88700832750
:104DF000C4FD88438327C4FDDE230347B4FD131697
:104E000007014182035784FD832644FDBE85029835
:104E1000AA872317F4FE8357E4FE3E85B25022543E
:104E200045618280011106CE22CC00102326A4FE0B
:104E30002324B4FEB2872313F4FE8327C4FE035752
:104E400064FEDAA38327C4FE032784FE98C3832766
:104E5000C4FE373700001307E74C98C78327C4FE0A
:104E60003737000013078775D8C78327C4FE03A808
:104E7000C7008327C4FE88438327C4FEDE2305477B
:104E80009306600B1306000EBE8502988327C4FEAE
:104E900003A8C7008327C4FE88438327C4FEDE23FC
:104EA00005479306F00F1306400FBE85029883272F
:104EB000C4FE03A8C7008327C4FE88438327C4FE1B
:104EC000DE23054781461306500FBE8502988327CF
:104ED000C4FE03A887008327C4FE88438327C4FE3B
:104EE000CE2309479386C182130680080298832740
:104EF000C4FE03A887008327C4FE88438327C4FE1B
:104F0000CE2309479386E1821306A00802988327DF
:104F1000C4FE03A887008327C4FE88438327C4FEFA
:104F2000CE230947938601831306C008029883277E
:104F3000C4FE03A887008327C4FE88438327C4FEDA
:104F4000CE230947938621831306E008029883271E
:104F5000C4FE03A887008327C4FE88438327C4FEBA
:104F6000CE230947938641831306000902988327BD
:104F7000C4FE03A887008327C4FE88438327C4FE9A
:104F8000CE2309479386618313062009029883275D
:104F9000C4FE03A887008327C4FE88438327C4FE7A
:104FA000CE230947938681831306400902988327FD
:104FB000C4FE03A887008327C4FE88438327C4FE5A
:104FC000CE2309479386A18313066009029883279D
:104FD000C4FE03A887008327C4FE88438327C4FE3A
:104FE000CE2309479386C18313068009029883273D
:104FF000C4FE03A887008327C4FE88438327C4FE1A
:10500000CE2309479386E1831306A00902988327DC
:10501000C4FE03A887008327C4FE88438327C4FEF9
:10502000CE230947938601841306C009029883277B
:10503000C4FE03A887008327C4FE88438327C4FED9
:10504000CE230947938621841306E00902980100C4
:10505000F240624405618280011122CE00102326B5
:10506000A4FE2324B4FEB2872313F4FE8327C4FED8
:10507000035764FEDAA38327C4FE032784FE98C384
:105080008327C4FE373700001307E74C98C78327F0
:10509000C4FE3737000013078775D8C70100724474
:1050A00005618280411122C60008938741BB23A27B
:1050B00007000100324441018280411106C622C42A
:1050C0000008138541BB31200100B2402244410158
:1050D00082801D7186CEA2CC80102326A4FA93076D
:1050E00004FB13062003BE85138541B3EFF03F8B0D
:1050F0002324A4FE832784FEF9C3232604FE55A897
:105100008327C4FA138747008327C4FE930604FF4E
:10511000B69783C707FCBE853A857D202322A4FE6F
:10512000032744FE85476311F7088327C4FABC3F71
:10513000A207C207C1873E878327C4FABC2FD98F35
:105140003E85EF1070732A878327C4FAF8C7832738
:10515000C4FADC3FA207C207C1873E878327C4FA8F
:10516000DC2FD98F3E85EF1030712A878327C4FA50
:10517000B8CB8327C4FAFC3FA207C207C1873E878A
:105180008327C4FAFC2FD98F3E85EF10F06E2A8753
:105190008327C4FAF8CB8327C4FA03C717028327EF
:1051A000C4FAA38CE70401008327C4FE85072326E5
:1051B000F4FE8327C4FE032784FEE3E3E7F4010043
:1051C000F640664425618280797122D60018232E2C
:1051D000A4FCAE87A30DF4FCFD572326F4FE832721
:1051E000C4FD9C4315476364F71C13972700B567FC
:1051F00093870783BA979C4382870347B4FD93073D
:10520000E00F631BF71A8327C4FD9C431387170025
:105210008327C4FD98C38327C4FD239207008327F7
:10522000C4FD239507008327C4FDDE2313871700E1
:1052300093160701C1820327C4FD56A33E87832727
:10524000C4FDBA970347B4FDD8ABBDA28347B4FDF4
:10525000C207C18389071397070141838327C4FDD0
:10526000FAA38327C4FD9C43138717008327C4FD3B
:1052700098C38327C4FDDE23138717009316070105
:10528000C1820327C4FD56A33E878327C4FDBA9776
:105290000347B4FDD8AB8327C4FD2386070005A2CE
:1052A0008327C4FDDE231387170093160701C182ED
:1052B0000327C4FD56A33E878327C4FDBA9703473F
:1052C000B4FDD8AB8327C4FDD8278347B4FDBA9774
:1052D00013F7F70F8327C4FDD8A78327C4FDDE2368
:1052E0003E878327C4FDFE2389076319F70C8327B4
:1052F000C4FD9C43138717008327C4FD98C37DA872
:105300008327C4FDDE231387170093160701C1828C
:105310000327C4FD56A33E878327C4FDBA970347DE
:10532000B4FDD8AB8327C4FD0347B4FDD8B78327AA
:10533000C4FD9C43138717008327C4FD98C341A075
:105340008327C4FDDE231387170093160701C1824C
:105350000327C4FD56A33E878327C4FDBA9703479E
:10536000B4FDD8AB8327C4FD9C4313871700832764
:10537000C4FD98C3A9A00347B4FD9307A00A631313
:10538000F7028327C4FDD8278327C4FDDC37631BBE
:10539000F7008327C4FD0547BAA78327C4FDBE27AE
:1053A0002326F4FE8327C4FD23A0070009A8832732
:1053B000C4FD23A0070021A0010011A00100832744
:1053C000C4FE3E85325445618280797106D622D46E
:1053D0000018232EA4FC232CB4FCB287231BF4FC5E
:1053E0008327C4FD035764FDDAA38327C4FD032785
:1053F00084FD98C38327C4FD373700001307E74CAB
:1054000098C78327C4FD3737000013078775D8C7AF
:10541000930700F8A307F4FE930700F8A307F4FE30
:105420008327C4FD03A8C7008327C4FD88438327BF
:10543000C4FDDE239306F4FE05472946BE85029887
:10544000C547A307F4FE8327C4FD03A8C70083272D
:10545000C4FD88438327C4FDDE239306F4FE05477D
:105460002546BE85029893071004A307F4FE832700
:10547000C4FD03A8C7008327C4FD88438327C4FD58
:10548000DE239306F4FE05472946BE8502980100F7
:10549000B250225445618280411106C622C40008E0
:1054A000EFE06FF2EFE01FB0EFD0BF93EFE00FC37C
:1054B000EFF0EF83EFD0BFD1EFF0DFBE1306000AAD
:1054C0009385418A138501C1EFF01F8BD146138666
:1054D00001C58145138501C1EFF0DF8E13068006FB
:1054E0009385C188138501C2EFF01FB735469385B8
:1054F000C188138501C3D13D1306C00E9385C188B1
:10550000138501C4EFF01F920100B2402244410113
:1055100082801D7186CEA2CCA6CACAC8CEC6D2C40D
:10552000D6C2DAC05EDE62DC66DA6AD88010232674
:1055300004FCEFE0BF972326A4FC1545EFE0DF9BBA
:10554000EFE0DF962326A4FC0325C4FCEFD05FB474
:10555000EFE08FBEEFF07FB69387C18BC44B93878C
:10556000018F03AB47019387419283AB4701938738
:10557000819503AC4701938701859C4F3E85EF10D1
:10558000103CAA8C2E8D93870185DC4F3E85EF1051
:10559000103B2A89AE89938701859C533E85EF1085
:1055A000103A2A8AAE8A93870185DC533E85EF1034
:1055B0001039AA872E880327C4FC3ACC3EC842CAB9
:1055C00052C456C64AC04EC26688EA886287DE86E2
:1055D0005A86A685B1671385877FEF20F06783C75A
:1055E0004184850713F7F70F2382E18483C7518431
:1055F000850713F7F70FA382E18483C761848507CA
:1056000013F7F70F2383E18483C74184858B93F7D6
:10561000F70F85C30145EFE07F800D45EFE01F8068
:105620001145EFE0AFFF1545EFE04FFF1945EFE003
:10563000EFFE03C751848D47B377F70293F7F70F57
:1056400081C70545EFE08FFD03C761849547B377B8
:10565000F70293F7F70FE38207EE0945EFE00FFC3F
:10566000E9BD3708100001117D183377B80026CA4C
:105670003378D80093D4450113D34601131E370065
:105680004EC61357D5010E089357D60193F4F47FF5
:105690001373F37F06CE22CC4AC893D9F50193DE6B
:1056A000F6013367C701131F350033E80701931F65
:1056B0003600338E64406380D9196356C013630487
:1056C000031CB70680009307F07F3368D800638F10
:1056D000F4369307800363C0C735FD4763CDC747E2
:1056E000130500023305C541B3D7CF01B316A80097
:1056F0003399AF00DD8E33392001B357C80133E948
:1057000026011D8F33092F41B3372F013306F74090
:105710009317860063D40724370780007D173374FE
:10572000E600630C042C2285EF10D042130785FF9E
:1057300093070002998FB357F9003316E400D18F15
:105740003319E9006341972A330597401306150082
:105750007D47634DC73813070002118FB356C90048
:105760003319E9003397E700558F33392001336946
:10577000270133D6C70081449377790081CF13770F
:10578000F90091476308F7001307490033392701EF
:105790004A963A899317860063D6071C138514002E
:1057A0009307F07FCE856304F520B70780FFFD17D0
:1057B000F18F9398D70113593900A607B3E8280150
:1057C000B1831375F57F9396C7005205F24062448A
:1057D000B182FE05C98ECD8ED2444249B24946857A
:1057E000B68505618280631E0E0A1383140013734D
:1057F000E37F63170322B367E701B368F801639D92
:10580000041A63870740638608443309FF41B307DE
:10581000074133362F013386C7409317860063D67E
:10582000074C3389EF41B307E84033B62F01338685
:10583000C740F68991B76350C00F6300030CB706E9
:1058400080009307F07F3368D800638AF43A9307A7
:10585000800363CBC713FD4763DFC73513090EFE13
:1058600093070002B3562801630AFE0013090004DF
:105870003309C94133192801B3EF2F013339F0013E
:105880003369D90031A2B367F801638A071C930713
:10589000FEFF638C07389306F07F6309DE1A3E8EA5
:1058A0000DBDB305934063910422B367E70163879D
:1058B00007329387F5FF638107449306F07F638C7B
:1058C000D520BE859307800363CCB72AFD4763CFFD
:1058D000B73C930700028D8F3319F700B356BF0012
:1058E000B317FF003369D900B337F0003357B7005F
:1058F0003369F9003308E84041ACB367F8016380CD
:1059000007349307FEFF638A07209306F07F63083E
:10591000DE2E3E8E2DBF631E0E149386140093F769
:10592000E67F63910734B367E7016395042C6380D6
:10593000073EB367F801638E07303309FF01B307F1
:105940000701333FE9013386E7019317860063D7E8
:105950000700B70780FFFD177D8E85449377790098
:10596000E39F07E09317D60193583900B3E8F80096
:10597000935736001307F07F638DE404B207B183B9
:1059800013F5F47FCE8581B53369F80133392001F1
:105990007A99B337E9013386E70093178600E3DF8E
:1059A00007FA85049307F07F6396F418CE851305F4
:1059B000F07F8147814801BDC1EB6384083A9316AB
:1059C00036009317D8018D82B3E8D700F689935734
:1059D0003800B3E7F800F9DB81451305F07FB7071E
:1059E00008008148CDB3370680FF7D167D8E937702
:1059F0007900998CE39507D8B5B74A85EF109015D3
:105A000013078501FD47E3D5E7D2130685FFB317DA
:105A1000C900014905BB3369F80133392001DDB103
:105A20003309FF413306074133342F0133048640E5
:105A30009317840063CD0724B3688900E39308CEED
:105A40008147814981441DBFE39808F80E059317EB
:105A5000D7010D81B3E8A700935737009DBF0E050E
:105A60009317D7010D81B3E8A700F284935737004D
:105A700011B73305934063820412B7068000930781
:105A8000F07F558F630DF32E9307800363CBA72020
:105A9000FD4763C3A72A93070002898F3319F700D4
:105AA000B356AF00B317FF003369D900B337F00026
:105AB0003357A7003369F9003A987E99B337F90153
:105AC000338607019A84D1BDB70680009307F07F23
:105AD000558FE319F3DE931736008D839318D801A1
:105AE000B3E81701F68993573800E5B5130715FE9B
:105AF0009306000233D7E700630AD600930600043A
:105B00003386C6403396C7003369C9003339200154
:105B10003369E9000146814491B53309FF01B307B8
:105B200007013336E9013E96931786008544E3D793
:105B300007E28944B70780FFFD17F18F135719005B
:105B400013791900336927019398F70133E9280184
:105B500013D6170015B113090EFE93070002B356B2
:105B60002801630AFE00130900043309C9413319EF
:105B70002801B3EF2F013339F0013369D90059B649
:105B80003369E7013339200133892F41B3B72F013E
:105B90003306F8409A84F689A5BEB367E7016382AD
:105BA00007189307F5FF6384071C9306F07F6304CF
:105BB000D5123E85D1BD93070002B387C741B31606
:105BC000F8003399FF0033D6CF01D18E333920014D
:105BD000B357C80133E926013E975DBB93173600E2
:105BE0008D839318D801B3E81701AE84935738001A
:105BF000F68949B3EDC33369F801E31F09DC0E05EB
:105C00009317D7010D81B368F50093573700D1B3CF
:105C10006381080E931636009317D8018D82B3E87E
:105C2000D700F6899357380091BB3309FF41B3077A
:105C30000741333F2F013386E7418544D1BC0E0530
:105C40009317D7010D81B368F500F284935737009D
:105C500015B30E059317D7010D81B3E8A70093572D
:105C6000370029BB9307F07FE382F6D43309FF01A5
:105C70003336E901B3070701B2979398F701135937
:105C8000190033E9280113D61700B684C1B9338946
:105C9000EF413307E84033B62F013304C740F6899C
:105CA00049B43369E7013339200101BD938705FE0B
:105CB00093060002B357F700638AD50093060004E9
:105CC000B385B6403317B700336FEF003339E001C7
:105CD0003369F90055BD931736008D839318D801A9
:105CE000B3E8170193573800EDB1B368C900E397E3
:105CF00008C68147814959B13389EF41B307E8406C
:105D000033B62F013386C740F689854411B4931604
:105D100036009317D8018D82B3E8D7009357380027
:105D2000B1B9931636009317D8018D82B3E8D70026
:105D3000AA84935738003DB9930705FE93060002E5
:105D4000B357F700630AD500930600043385A640D5
:105D50003317A700336FEF003339E0013369F900DF
:105D6000A9BB81451305F07FB7070800A9BC33091B
:105D7000FF01B30707013336F9013E9675B3931659
:105D800036009317D8018D82B3E8D70093573800B7
:105D900089B1397193D7450122DC4AD856D22A8974
:105DA0001394C50006DE26DA4ED652D45AD05ECE03
:105DB00013F5F77F318093DAF501630B0510930734
:105DC000F07F630BF514135AD9010E0433648A0073
:105DD000370A8000336A4401131B3900930415C04D
:105DE0000144814B13D846011399C6001378F87FFC
:105DF000B2881359C90093D9F601630E08089307B6
:105E0000F07F6300F8041357D6010E0933692701A8
:105E1000130818C0B70780003367F90093183600DD
:105E2000B38404418145BD4733C83A0163E4871A0E
:105E300097770000938787A10A043E9410403E960E
:105E400002863367C90093841480631207101364B9
:105E5000240081488945C1BF1306F07F814701476F
:105E6000B207F25062545206B1837E08D18FB3E775
:105E70000701D2544259B259225A925A025BF24B4C
:105E80003A85BE852161828001481306F07FB707FD
:105E900008000147F1B73367C9004DC763080930EF
:105EA0004A8532C4EF10004B2246130755FFF547D1
:105EB000930685FF998F3319D900B357F60033E75E
:105EC0002701B318D60026959304353F8145A1BF1D
:105ED000336A240163030A0636C632C46306042A01
:105EE0002285EF1020472246B246AA84130755FFA9
:105EF000754A138B84FF330AEA4033146401335A22
:105F00004901336A8A00331B69011305D0C0B30409
:105F100095400144814BF9B5336A240163180A00A6
:105F20002144014B9304F07F894B6DBD228A4A8B3B
:105F300031449304F07F8D4B75B51144014B81447E
:105F4000854B4DB51364140081488545E9BD136444
:105F500034004A878D45C1BD630A052E8547898F68
:105F60009306800363DDF632014681470147CDBDCC
:105F7000CE868947638DF53A8D47E387F5F08547EF
:105F80003688E383F5FE1385F43FE357A0FC93F7CF
:105F900078006396072893D638009317770063D864
:105FA0000700B70700FFFD177D8F13850440930797
:105FB000E07FE3C3A7EA1316D70193179700B183D5
:105FC0003367D6001376F57F61BDD6865287DA88AF
:105FD000DE8545B763614723630DEA20DA86FD1449
:105FE0005284014B9317870013D388013363F30066
:105FF000935E0301B357D403131F0301135F0F0113
:1060000093D50601139E88003374D4033307FF022F
:106010004204C18D63FBE5009A951386F7FF63EE9A
:10602000652663FCE526F9179A95998D33D7D50334
:10603000C206C182B3F5D5033306EF02C205D58D82
:1060400063FBC5009A959306F7FF63E6652463F446
:10605000C52479179A95C20741645D8F9307F4FFB1
:106060003375F70093580701935F0E01B377FE0075
:10607000B302F502B386C540B383F80293D502019B
:106080003386AF021E962E963385F803637376002F
:106090002295C168FD189355060133761601420614
:1060A000B3F81201AA95469663E6B6126382B61259
:1060B0003306CB408D8E333BCB00338B664113854B
:1060C000F43F630C6317B358DB0393550601337B2E
:1060D000DB03B3061F03420B33EB6501637BDB007D
:1060E0001A9B9385F8FF636D6B20637BDB20F918A7
:1060F0001A9B330BDB40B356DB0342064182337BF2
:10610000DB03330FDF02420B33666601637BE6017C
:106110001A969385F6FF6367661E6375E61FF91688
:106120001A96C208B3E8D8009395080193D20801E3
:10613000C181B38EF5023306E641B385BF0293D623
:106140000E01B387F202BE95AE96B38F5F0263F481
:10615000F600C167BE9FC165FD1593D70601ED8EA0
:10616000C206B3FEBE00BE9FF696637FF6091A967E
:106170009387F8FF6369661A6368F619630FF61B65
:10618000BE8893E8180011B54A85EF10A01C1307CC
:106190005501F145930405022246B246E3DAE5D4FF
:1061A000130485FF331A8900014B85B3328532C44D
:1061B000EF10401A13075501F146AA87224613052E
:1061C0000502E3D6E6CEE1173317F6008148E5B9BC
:1061D000E370CBEE729B3335CB011A95AA9613056B
:1061E000F7FF6378D30263E6B6106382D5102A877F
:1061F000C1B5E3651BDF93551B009316FA011354D9
:106200001A00CD8E7E0BF9BBE31DF6F7E38F06D6A1
:10621000B9BFE31ED3FCE378CBFD2A8751BD93F7CA
:10622000F8009146E389D7D693B7C8FF9386480014
:1062300093C717008D823E978DB381468547E34C07
:10624000A0FEFD58E31C05D0930410C085471385BC
:10625000E441B316A70033D6F8003395A800D18ED9
:106260003335A000C98E13F676003357F70001CE00
:1062700093F7F60011466388C70093874600B3B6CC
:10628000D7003697BE869317870063D80704054664
:1062900081470147F1B636877DBBB28779B3FD46AA
:1062A000E3D7F6FA0556098E930600023356C70067
:1062B0006388D7009387E443B317F700B3E8F80087
:1062C000B3361001D18E13F67600814701CE93F7D5
:1062D000F60011460147E392C7FA93179700131689
:1062E000D701B18313D73600518F014695BEE370B5
:1062F000CBF0729B3335CB011A957917AA964DBB1B
:10630000AE88C5BBAE8631BD93171E0033BEC70134
:1063100072931A96F9183E8EE315F6E7E307DEC688
:1063200093E818009DB1BE88E30AF6FF99BD368850
:106330001306F07F8147014725B6E367DEFCBE8880
:10634000E310DEFE99B139714AD813D945014ED612
:1063500052D456D29399C50006DE22DC26DA5AD0F2
:106360005ECE1379F97F2A8A93D9C90093DAF501B1
:10637000630D090E9307F07F6306F9181354D501D6
:106380008E09B36934013704800033E48900931423
:106390003500130919C08149814B13D74601139A5F
:1063A000C6001377F77FB285135ACA0013DBF601D4
:1063B000630B07109307F07F6303F7049357D6012D
:1063C0000E0A33EA4701130717C0B7078000B36707
:1063D000FA00931536003A99814833C76A01BD46E1
:1063E0003A851308190063E836171766000013068C
:1063F000E6498A09B29983A60900B2968286B367F4
:10640000CA001309F97F6399071293E929008145AE
:106410008948E1B701479307F07F370408008144BA
:106420003204D20731807E075D8C598CA285F250F0
:10643000625426854259D254B259225A925A025B6A
:10644000F24B216182805A853E84AE84C68B894797
:10645000638DFB0E8D47E38FFBFA85472A87639E8A
:10646000FB3881470144814465BF33E4A90061C022
:1064700036C632C4638C092A4E85EF00B06D2246C1
:10648000B246AA87130755FF7544938487FF198C7A
:10649000B399990033548A0033643401B3149A00D9
:1064A00013D746011309D0C0139AC6001377F77F9C
:1064B0003309F9408149814BB285135ACA0013DB75
:1064C000F601E31907EEB367CA00B1C7630F0A22EA
:1064D000528532C4EF00106822462A87930655FF82
:1064E000F547930587FF958F331ABA00B357F60027
:1064F000B3E74701B315B6003309E9401309D9C022
:106500008148E1BD33E4A90001ECA14981441309AC
:10651000F07F894B59B593E919008145854875BDD0
:106520004E84AA84B1491309F07F8D4BBDB59149C2
:1065300081440149854B95B593E93900D2878D484F
:1065400069BD89475685E397FBF02A879307F07F5B
:1065500001448144F1B5C16E1386FEFF93D6040158
:1065600013DE0501F18CF18D338695023383B6027B
:106570009358060133059E021A95AA98B382C60362
:1065800063F36800F692C16F1383FFFF33F5670072
:1065900093D30701B3F76800C207337366003E93D5
:1065A0003306950293D80801B387A602135F06014C
:1065B000B3849302BE94FA94B38E760263F3F4002C
:1065C000FE9E416A9307FAFF935F0401B376F400DD
:1065D000B3F9F4007D8EC1803384D502C209338FB4
:1065E000D401B299CE98B307DE02935E0401B3855D
:1065F000BF02AE97BE9E330EFE0363F3BE00529EF3
:10660000C1679385F7FF33F6BE006D8C4206229674
:1066100093DE0E01B305D502769E3385AF0213D407
:106620000501B386D302AA96A296B38FF30363F350
:10663000A600BE9F41657D15B3F7A600C2076D8D0C
:10664000AA97B3855800B3B93501FA97B295338448
:10665000370133B6C500B30EC4013385CE003334E1
:106660003401B3B7E701C18F33BECE0113D40601A5
:106670003336C5003E943366CE0093949500329431
:106680007E94B3E46400260493567501B3349000FD
:10669000DD8193179500CD8C558CDD8C931774009C
:1066A00063DB070093D7140085889316F401DD8C13
:1066B000D58C058042899307F93F6359F00893F61A
:1066C000740081CE93F6F40011466388C600938669
:1066D0004400B3B496002694B6849316740063D82D
:1066E0000600B70700FFFD177D8C9307094093064E
:1066F000E07F63CFF60E93D634009314D4012604C2
:10670000D58C318093F7F77F21BB328532C4EF00FF
:10671000704493065501F147130705022246E3D161
:10672000D7DC6115B317A6008145F9B3EF0090429D
:1067300013075501F145930705022246B246E3D5FA
:10674000E5D461153314AA00814499BB85469D8E1A
:10675000B1E71309E941B3972401B3D4D400331945
:106760002401B337F000B3649900DD8C93F7740013
:10677000B356D40081CF93F7F40011466388C70065
:1067800093874400B3B49700A696BE84939786007F
:1067900063D8070485470144814459B11306800337
:1067A000E341D6CC7D46E356D6FA0556B307F6400C
:1067B000930500023356F4006387B6001309E943DA
:1067C000B3172401DD8CB3349000D18C93F67400A0
:1067D000014499CA93F7F40011468146E392C7FA3F
:1067E000139496003180F6068D80D58C81470DB9C3
:1067F0009307F07F0144814425B142896DBD37077D
:1068000010007D1701113373B70093D84601758FBF
:10681000935ED60122CC26CA0E0393D4450193572A
:10682000D5010E0706CE4AC84EC693F8F87F130E60
:10683000F07F33E7EE0093F4F47F13D4F50133E3F4
:106840006700131F3500FD82931E36006380C81950
:1068500093C61600B38514416305D4126351B01872
:10686000638B081AB70780005D8F6380C459930754
:10687000800363C3B734FD4763C4B748930700027E
:106880008D8FB3D9BE003318F700B39EFE00336876
:1068900038013357B700B339D001336838013303B7
:1068A000E340B3090F41B3373F013306F340931779
:1068B000860063D30724370980007D1933792601C8
:1068C000630F092C4A85EF00F028130785FF930713
:1068D0000002998FB3D7F9003316E900D18FB3992D
:1068E000E9006344972A058F13061700FD4663C429
:1068F000C63A13070002118FB3D6C9003398E900D6
:106900003397E700558F33380001B369070133D659
:10691000C700814493F7790081CF93F6F90091473E
:106920006388F6009386490033B836014296B689EB
:106930009317860063D6071C138714009307F07F14
:1069400005886306F720B70780FFFD17F18F1398BE
:10695000D70193D93900A60733683801B18313777B
:10696000F77F9396C7005207B1827E04D98EC18EFD
:10697000F2406244D2444249B2494285B68505613B
:1069800082806356B00A638A0812B70780005D8F61
:106990006386C42D9307800363C7B718FD4763D18F
:1069A000B73C138805FE93070002B3590701638AB9
:1069B000F50093070004B385B7403317B700B3EE73
:1069C000EE003338D0013368380195A2B367D701A0
:1069D0009385148099E393C61600630AD404D1E129
:1069E0009387140093F7E77F6398071EB367E3016B
:1069F0003368D701639204166381073C631508422C
:106A0000131835009316D3011358380033E80601E4
:106A10009357330019A2B367D7016384071A93878A
:106A2000F5FF638A073A638BC523BE8589B56398F2
:106A3000051C9386140093F7E67FC1EFB367E3016B
:106A4000639F0434638C0744B367D701639307469D
:106A50000E051318D3010D813368A8009357330036
:106A60006DA8B385984063960420B367E301638CF7
:106A700007309387F5FF638807401305F07F638233
:106A8000A520BE859307800363C1B72AFD4763C76E
:106A9000B73C930700028D8F3318F3003356BF00C5
:106AA000B317FF003368C800B339F0003353B300A5
:106AB0003368380133076740ADACB367D7016382F1
:106AC00007109387F5FF638E071E638FC52DBE8564
:106AD000D1B59307F07F638BF606FA9E33B6EE01CD
:106AE000B307E300B2971398F70193DE1E00B36972
:106AF000D80113D61700B68493F77900E39F07E017
:106B00009317D60113D839003368F800A685935738
:106B100036001307F07F6380E506B207B18313F7F1
:106B2000F57F05883DBD3367D7013338E000B309F1
:106B3000E801B3B7E9013386670093178600E3DD08
:106B400007FA85049307F07F639BF4180588130701
:106B5000F07F8147014831B5639007106300083C1E
:106B6000131836009317D701135838003368F8000C
:106B7000368493573700B367F800E9DB0144130705
:106B8000F07FB70708000148E9BB370680FF7D1694
:106B90007D8E93F77900998CE39107D895B74E8550
:106BA000552F13078501FD47E3D3E7D2130685FF71
:106BB000B397C900814935B33368D7013338000131
:106BC000CDB1131835009317D3011358380033682B
:106BD000F8009357330035BFB309DF413309E34071
:106BE00033363F013309C9409317890063CA072030
:106BF00033E82901E31608CC8147014439BFB38546
:106C0000984063810414B70680009307F07F3363D4
:106C1000D3006381F8209307800363CCB722FD473C
:106C200063C9B72C930700028D8F3318F300B35656
:106C3000BF00B317FF003368D800B339F0003353F7
:106C4000B300336838011A97B309D801B3B7D90133
:106C50003386E700C684D5B5E31208F21318350071
:106C60009317D301135838003368F8009357330053
:106C700019B7370580009307F07F3363A300E393D0
:106C8000F8E00E061318D7010D823368C800935739
:106C900037003684CDB505179306000233D7E700D9
:106CA000630AD600930600043386C6403396C700B5
:106CB000B3E9C90033383001B369E80001468144C3
:106CC00025BDB309DF01B307E30033BFE901338614
:106CD000E701931786008544E3D007E28944B707AC
:106CE00080FFFD17F18F13D7190013F819003368CF
:106CF00007019399F701B3E9090113D6170019B9F0
:106D0000138805FE93070002B3590701638AF50053
:106D100093070004B385B7403317B700B3EEEE0016
:106D20003338D00133683801ADBE3363E301333803
:106D30006000B3890E41B3B73E013306F740C68405
:106D40003684B5B6B367E301638707189387F5FF09
:106D5000638C071C9306F07F638ED50ABE8565BDE4
:106D6000930700028D8FB3D9BE003318F700B39E8E
:106D7000FE00336838013357B700B339D0013368A8
:106D800038013A936DB3131836009317D70113588F
:106D9000380033E807013684935737009DBBBDCBDD
:106DA0003367D701E31C07DC0E051318D3010D81EF
:106DB0003368A800935733007DBBE30F08E2131834
:106DC00036009317D701135838003368F80036841B
:106DD0009357370099B3B309DF41B307E340333F1B
:106DE0003F013386E7418544D9B413183500931623
:106DF000D3011358380033E8060193573300A5BB7D
:106E0000B389EE413306674033B93E013309264169
:106E100036847DB40E061318D7010D823368C8007E
:106E20009357370089BBB309DF41B307E3403336DB
:106E30003F013386C7409317860063D7070AB3899B
:106E4000EE41B3076740B3BE3E013386D741368477
:106E5000D1B43363E30133386000FDB3138805FE1A
:106E600093070002B3590301638AF50093070004F6
:106E7000B385B7403313B300336F6F003338E0018D
:106E8000336838017DB5B389EE41B3076740B3BEBF
:106E90003E013386D7413684854411BC1318360031
:106EA0009317D701135838003368F8009357370009
:106EB000ADB1B309DF01B307E30033BFE9013386A6
:106EC000E70193178600E3D907C2B70780FFFD17D4
:106ED0007D8E854415B10E061318D7010D823368D7
:106EE000C8009357370035B133E8C900E30608D02E
:106EF00021B1138805FE93070002B3590301638A89
:106F0000F50093070004B385B7403313B300336F24
:106F10006F003338E001336838013DB30144130793
:106F2000F07FB707080035BCB309DF01B307E30002
:106F3000B3BED9013386D70169BB93D74501B706E4
:106F400010001387F6FF93F7F77F1306E03F6D8F6E
:106F5000FD81635CF6001306D041635AF6003705E5
:106F600000801345F5FF2E9582800145828013062F
:106F700030431D8E7D48558F635DC80093063041B8
:106F8000B387F640B357F7003305F040E5F13E858F
:106F900082809387D7BEB317F7003355C500C98FDA
:106FA000E5B7411106C622C426C205CD9357F54167
:106FB000B3C4A7009D8C2A842685692E9306E041E0
:106FC000898EA9477D8093F6F67F63CDA7022D4772
:106FD000098FB3D7E4005505B207B394A400B18379
:106FE00029A00144814681478144B207D206B1837A
:106FF0007E04D58FC18FB24022442685BE8592443F
:10700000410182805515B397A400B207B183814432
:10701000E9BF15CD411122C406C62A84252E930648
:10702000E041898EA94793F6F67F63DCA7025515E8
:10703000B317A400B207B1830147B2402244B2079C
:10704000D206B183D58F3A85BE85410182808147C2
:107050008146B207D206B1830147D58F3A85BE85F6
:1070600082802D47098FB357E400B20713075501FB
:107070003317E400B183D1B7411106C622C426C23A
:107080000DCD9357F54133C4A7001D8CAA842285EA
:10709000D1249307E0093387A74093076009FD8057
:1070A00063CCE702A1469377F70F63D5A60061157D
:1070B0003314A4002604258021A081448147014483
:1070C000260413559400B2402244DE07FE045D8D71
:1070D000458D9244410182809307900963DDE7006A
:1070E0009307B5019546B317F400898E3354D40045
:1070F000B337F0005D8C954763D6A7009307B5FFC3
:107100003314F400B70600FCFD1693777400337651
:10711000D40085C39377F4009145638CB7001106C2
:107120009317560063D707009307F009758E3387CE
:10713000A7401314660025809377F70F51B71357B4
:1071400075011377F70F41119307170022C426C268
:107150001314950006C693F7E70F25809354F501A5
:1071600085C793573400130707387604B2075207D0
:10717000B1831395F401D98FC98FB240228522447F
:107180009244BE854101828005EB39C42285D92213
:10719000A94763C6A7042D47098F930755013357A5
:1071A000E4003314F4009317C70013079038098FD5
:1071B000B1831377F77F5DBF01CC13573400B70756
:1071C0000800D98FB2077604B1831307F07F79BF27
:1071D0001307F07F814759BF0147814741BF13071C
:1071E00055FF3317E40001447DBF93D645019397C3
:1071F000C50093F6F67FB183138616008E071357EA
:10720000D5011376E67FFD815D8F9318350035CE6D
:10721000138806C89307E00F63DD070181471395C4
:1072200097009306F00FDE062581FE05558D4D8DE6
:1072300082806355000B931765000E07B337F0008B
:10724000D98F93D8D801B3E7170113F777006301FB
:10725000071013F7F70091466303D700910737072C
:1072600000047D8F75C7130718001306F00F93767F
:10727000F70FE305C7FA9A07A58313959700DE0673
:107280002581FE05558D4D8D8280B367170199EEDE
:1072900085CF95479A07A5831395970093F6F60F28
:1072A000DE062581FE05558D4D8D8280A5DBB70755
:1072B0004000139597009306F00FDE068145258167
:1072C000FE05558D4D8D828081471395970081462F
:1072D000DE062581FE05558D4D8D8280A5576348BC
:1072E000F804F94737068000B38707417D45598E7A
:1072F0006351F504795733070741130500023357EB
:10730000E6006388A700938626CAB316D600B3E8C2
:10731000D800B3371001D98F13F77700014815FB58
:10732000139757008546E34807F48146A5B7814681
:107330008DB7938626C83397D8003337E000B3164D
:10734000D600B3D8F800B367D700B3E7F800E9B7C1
:10735000C28689B7C167637CF5029307F00F1307F4
:10736000000263EBA7009757000093872756AA9760
:1073700088233305A7408280218197570000938797
:10738000E754AA97882361473305A7408280B7074F
:107390000001636DF50061819757000093870753E3
:1073A000AA97882321473305A740828041819757B8
:1073B00000009387A751AA97882341473305A74028
:1073C00082809387C180AA8588439DA29387C180CC
:1073D000AA85884355A8B3C7A5008D8B3307C50080
:1073E00081E78D4763EDC700AA87637EE508942196
:1073F00085078505A38FD7FEE3EBE7FE82809376B2
:107400003500AA8789CA942185078505A38FD7FEF1
:1074100093F63700C5BF9376C7FF138606FE63F069
:10742000C70683A3050083A2450083AF850003AF91
:10743000C50083AE050103AE450103A3850183A802
:10744000C5019385450223A0770003A8C5FF23A2A9
:10745000570023A4F70123A6E70123A8D70123AAF5
:10746000C70123AC670023AE17019387470223AE01
:1074700007FF75B790419107910523AEC7FEE3EB77
:10748000D7FEE3E6E7F68280DDC183A7C5FF4111A1
:1074900022C406C626C21384C5FF63D307003E94E8
:1074A000AA84EF30805C938781849C4381EF232200
:1074B000040023A481842244B240268592444101E1
:1074C0006F30C05A637EF40014403307D4006396D3
:1074D000E7009843DC43369718C05CC0D9BFBA8731
:1074E000D84319C3E37DE4FE94433386D700631F7A
:1074F00086001040B29694C33386D700E31DC7FAC6
:1075000010435843B29694C3D8C375B76375C4008B
:10751000B1479CC04DB71040B306C4006316D700F6
:1075200014435843B29614C058C0C0C369B7828090
:10753000011126CA93843500F19806CE22CC4AC8A0
:107540004EC6A104B14763F5F404B14463E4B40446
:107550002A89EF3080519387818498433A8429E4C3
:107560009387C1849C4399E781454A85EF00F07277
:1075700023A6A184A6854A85EF003072FD596319C0
:107580003507B1472320F9004A85EF30204E29A066
:10759000E3DE04FAB1471CC10145F2406244D24423
:1075A0004249B249056182801C40858F63CF070242
:1075B000AD4663F6F6001CC03E9404C031A05C40AA
:1075C0006313870223A4F1844A85EF30204A130510
:1075D000B4009307440061993307F5405DDF3A94A6
:1075E000898F1CC05DBF5CC3C5B72287404085BF83
:1075F000130435007198E30285FCB305A4404A8565
:10760000EF00B069E31B35FBADBF797122D44AD0DE
:1076100052CC56CA5AC806D626D24ECE3A8AAE8A1E
:1076200032843689428B0147635806003707008051
:107630003344C7001307D00298A393F4F8FD9307CF
:1076400060048D466388F400930750048946639371
:10765000F4000509DA879308C100130881004A87FE
:10766000D6852286EF10D06193077004AA896396AD
:10767000F400137A1A00630A0A0493076004338A39
:1076800029016397F40203C7090093070003631EEF
:10769000F700014681465685A285EF40B02A11C504
:1076A00085473389274123202B0183270B003E9AEE
:1076B000014681465685A285EF40D02811E152C689
:1076C00013070003B24763E24703B2474257B25081
:1076D0002254B38737411CC34E8592540259F24954
:1076E000624AD24A424B456182809386170036C671
:1076F00098A3C9BF10A1130725009307B00263D652
:107700000500B305B0409307D0021CB1A54763DA6A
:10771000B70441119307F100BE88294813033006CE
:10772000B3E605031386F7FF93860603A38FD7FE00
:10773000B3C60503634DB30093860603F917A30F81
:10774000D6FE63E917013305A74041018280B28765
:10775000B685F9B7850783C6F7FF0507A30FD7FEE0
:10776000CDB79307000313074500938505033CA19C
:107770002CB13305A740828019713ACE86DEA2DC97
:10778000A6DA2E84CAD8CED6D2D4B689DAD0DECE46
:10779000E2CC3289D6D2E6CAEAC8EEC6AA84EF3075
:1077A000A026832B05005E85EF00F056032B040016
:1077B000724702DC93760B102A8C034A84011C4327
:1077C000F1CA9386470014C39C43081098433AD0EB
:1077D000D8433AD298473AD4DC473ED6EF40F056E9
:1077E00028C46CC4832CC404175700001307071E59
:1077F000832A8404032D0700832D470093971C00E0
:1078000085836A86EE865685BE853ECEEF40703013
:1078100041EDF2476A86EE865685BE85EF4010241C
:107820006354A008014681465685E685EF40102343
:10783000635605009307D002A301F4049307700474
:10784000975A0000938A0A1963F64701975A000075
:10785000938A8A18137BBBFF8D47232064011CC8C1
:10786000014B4E87CA867018A2852685C12EFD5C05
:10787000631E95157D55F6506654D6544659B65933
:10788000265A965A065BF64B664CD64C464DB64D7C
:10789000096182809D07E19B9386870014C398430A
:1078A000DC4338C47CC43DBF5686E6865685E685F3
:1078B000EF40302611CD93077004975A0000938A49
:1078C000EA11E3F947F9975A0000938A6A1159B708
:1078D0005C407D57137DFA0D6395E70899475CC0BE
:1078E000544013670B403C18D6853EC018C0930720
:1078F000310302C2D2881308410366862685EFF061
:10790000DFD093077004AA8AD255631BFD00F55798
:1079100063C5F5005C4063D8B708791A137AFA0F8B
:107920009307500663E64705FD15528613050405C7
:107930002EDAEFF03FDC625785462A8BB307A700AB
:107940001CC863C5E6001840058B19C385071CC811
:1079500083473103E38707F09307D002A301F404C0
:1079600009B713077004E31DEDF6BDFB854785BF1E
:1079700093076006631BFA025C40635BB0000CC8AF
:1079800081E71840058B09CF8507AE971CC809A869
:1079900089E718408546058B19C39386270014C8CC
:1079A0002CCC014B75B7130A7006E25763C9F5007A
:1079B0001C400CC8858BEDD793871500C1BF0547C8
:1079C0006344B00009470D8FBA97C9B71C4013F73D
:1079D000074015E314485686CA8526858299E30B2D
:1079E00095E91C40898B63960724F2574844E35479
:1079F000F5E83E8549B513075006637B47192844CF
:107A00006C4401468146EF40E07339E985461756DC
:107A10000000130626FDCA8526858299E30C95E5AC
:107A20005257E2576345F7001C40858BDDDBE28649
:107A30005E86CA8526858299FD57E30DF5E2014AE7
:107A4000930AA4017D5BE257FD17E35CFAF88546D3
:107A50005686CA8526858299E30E65E1050AE5B753
:107A6000D2576346F006854617560000130686F780
:107A7000CA8526858299E30F95DFD2576257D98F41
:107A800081E71C40858BB1DFE2865E86CA8526854C
:107A90008299FD57E300F5DE014A130BA401FD5B5B
:107AA000D257B307F040634BFA00E2565686CA85B8
:107AB00026858299FD57E316F5F26DBB85465A86F9
:107AC000CA8526858299E30775DB050AD1BF3C4C40
:107AD000625A63D347013E8A635A4001D286568672
:107AE000CA8526858299FD57E306F5D8814C130D8A
:107AF000A401FD5D09A885466A86CA852685829906
:107B0000E30AB5D7850C032B8405D28763530A009B
:107B10008147B307FB40E3C0FCFE5257E257634D79
:107B2000F7021C40858B8DEBE2575257338AE740B2
:107B30006344EB00338A6741635B4001D28633863E
:107B40006A01CA8526858299FD57E305F5D2814AE7
:107B5000130BA401FD5B15A0E2865E86CA8526850F
:107B60008299FD57E312F5FC31B385465A86CA85E2
:107B700026858299E30075D1850A5257E257998F7D
:107B8000528763530A000147998FE3C0FAFE91BD03
:107B9000E25605476344D700858BB5C785465686B0
:107BA000CA85268582997D5AE30645CDE2865E86A2
:107BB000CA8526858299E30F45CB28446C4401464B
:107BC0008146EF4020581DC9E25613861A00CA8527
:107BD000FD1626858299E30F45C9DA86130604054A
:107BE000F9B585465686CA8526858299E30475C906
:107BF000050AE257FD17E346FAFEC5B7014A930AA4
:107C0000A401FD5BFDB785465686CA852685829907
:107C1000E31595FD85B185465686CA8526858299E8
:107C2000E30A65C5050A5C447257998FE345FAFE7D
:107C30006DBB014A930A94017D5BF5B7797156CA11
:107C40009C49BA8A984522D426D24ECE52CC06D62A
:107C50004AD05AC85EC6AA892E84B284368A63D3B3
:107C6000E700BA879CC00347340419C385079CC04A
:107C70001C4093F7070281C79C4089079CC00329D9
:107C8000040013796900631A0900130B9401FD5B6A
:107C90005C449840998F634CF9041C40834634043B
:107CA00093F70702B336D000A5EB13063404D28550
:107CB0004E85829AFD576303F5041C401146984097
:107CC000998B544481446397C700B384E64063D3DF
:107CD000040081441C4418486354F700998FBE94F3
:107CE000014969047D5B63982405014509A885461F
:107CF0005A86D2854E85829A631E75017D55B25093
:107D0000225492540259F249624AD24A424BB24B2F
:107D1000456182800509ADBF3307D4001306000317
:107D2000A301C7040347540493871600A29789064A
:107D3000A381E7049DBF85462286D2854E85829A1F
:107D4000E30E65FB050945B7797122D426D24AD0E6
:107D50004ECE06D652CC56CA5AC8B689942D930731
:107D600090063289AA842E8413863504638DF60228
:107D700063E2D706930780056387F61863EDD700A3
:107D8000638F062093073004638FF60A930A240456
:107D90002301D404D1A0930730066386F60A930723
:107DA0004006E395F6FE1C40084393F6070893054A
:107DB0004500CDC61C410CC363D807001307D00291
:107DC000B307F040A301E404975600009386C6C1B0
:107DD00029476DA8930700076383F61663E5D7026A
:107DE0009307E006638AF6189307F006E390F6FA25
:107DF0000C401C4313F80508138547006308080668
:107E000008C39C438DA893075007E383F6FE9307AE
:107E10008007638AF61293073007E399F6F61C434E
:107E2000D04181459386470014C383AA0700568535
:107E3000EF20304201C53305554148C05C401CC8A5
:107E4000A301040461A81C43930A240493864700F9
:107E50009C4314C32301F4048547D5B793F6070464
:107E60001C410CC3B1DAC207C187B9B793F5050449
:107E700008C3C1D99E231307F0066387E60E975601
:107E80000000938666B62947A30104044C400CC445
:107E900063C5050008406D9908C099E3B28A89CD91
:107EA000B28AB3F5E702FD1AB6958C212380BA0099
:107EB000B3D5E70263F0E70CA147631EF7001C404F
:107EC000858B91CB58401C4863C7E700930700039C
:107ED000A38FFAFEFD1A3306564110C84E87CA8694
:107EE0007000A2852685EFF07FD57D5A631D450B76
:107EF0007D55B250225492540259F249624AD24AF4
:107F0000424B45618280A382D50497560000938638
:107F1000A6AD0C40084313F805081C411105630D7C
:107F2000080208C313F7150001C793E505020CC04A
:107F30004147B9FB0C4093F5F5FD0CC0B1B79C412E
:107F400093E707029CC193078007A302F4049756A6
:107F500000009386A6AA75BF13F8050408C3E303BF
:107F600008FCC207C1837DBF975600009386C6A751
:107F7000214719BFAE8735B794411C43CC4913F84C
:107F80000608138547006306080008C39C438CC39A
:107F900039A008C393F606049C43F5DA8EA3232880
:107FA0000400B28A25BF14485686CA852685829960
:107FB000E30045F51C40898B8DE7B2474844E35AFE
:107FC000F5F23E853DB785465686CA852685829957
:107FD000E30065F3050A5C443247998FE345FAFEF6
:107FE000E9BF014A930A94017D5BF5B79C451D7179
:107FF000A2CCCEC6DAC066DA86CEB28CA6CACAC811
:10800000D2C4D6C25EDE62DC6AD86ED61386F7FFB3
:108010001307C015368BAA892E8481466377C70063
:10802000938637EA9307D0159CC51C40930AC40178
:10803000D68493E707781CC00149814D014C014A61
:10804000014D814B13069004130800708548930E70
:1080500000400943130E50061D4F184415CB83A74B
:108060000C009C23638BC7126368F60C9305900386
:1080700063E4F50A9305100363FBB7149305D0027C
:108080006382B71663E3F5041307B002638CE71449
:1080900063060D001C4093F7F7EF1CC0FD1D8547DC
:1080A00063E9B72163EC9A1E0549F64066444A85A8
:1080B000D6444649B649264A964A064BF25B625C6C
:1080C000D25C425DB25D256182809305E002638EE1
:1080D000B71493050003E39DB7FA0C4013F50510A0
:1080E0007DC593F5F5F70CC0050D81C60507FD1696
:1080F00018C41C44FD171CC41C4885071CC883A752
:108100004C00FD1723A2FC006355F01683A70C005A
:10811000850723A0FC0091B7130750046381E71281
:1081200013076004638AE70E13071004E392E7F66F
:10813000E3901DF7894D65A06383C7116361FE0459
:1081400013074005638EE70C6364F7021307E0042E
:10815000E390E7F463900D0A63100D0A18409375DD
:108160000770639B05091377F78718C0854D85A8AD
:10817000130790056389E7041307100645BF13072B
:10818000E006E389E7FC6368F7021307600663858E
:10819000E70813079006E39DE7EE63180906E31B63
:1081A0000DEE184093750770E39A05EF1377F78784
:1081B00018C005492DA0130740076383E70613077E
:1081C0009007E397E7ECE315E9ED214909A8338728
:1081D0002D01E31F07EA18401377F7E718C09CA0AA
:1081E000850401BF184093750708E38305EA1377F8
:1081F000F7F7EDB7638D6D06630519011147E319B4
:10820000E9E805091379F90FD9BF1307D9FF1377E7
:10821000D70FE31F07E6F5B7E31C69E60D49C1B7C1
:108220001947E317E9E61D495DBF1840937507201C
:10823000E38005E61377F7D718C0EA8B4DB71840EF
:10824000937507506388D50193750740E38205E471
:10825000E3060DE49375072081E5330A7D41268C02
:108260001377F7871367071818C0014D8DBF8D4D21
:10827000BDB783270418E6854E8536C68297B24679
:1082800013069004130800708548930E00400943BC
:10829000130E50061D4FE30205DCDDBBFD148327E2
:1082A000C4178C2066864E8582971C48FD171CC813
:1082B000D5BB9307F9FF19476366F7028947A68D77
:1082C00063FF2707330799401377F70F8D46B3876E
:1082D000ED0093F7F70F63EBF60275191379F90FB9
:1082E000B38424411C4013F7071051CF93F7074084
:1082F000B1CBE3FB9ADAFD148327C4178C20668682
:108300004E8582971C48FD171CC8E5B7FD1D8327C5
:10831000C41783C50D0066864E853AC682971C48F1
:108320008D463247FD171CC85DB7FD148327C4175F
:108330008C2066864E8582971C48FD171CC8E3E694
:108340009AFE9DB31C4883C5F4FF1389F4FFFD1703
:108350001CC8930750066382F50293075004638E8E
:10836000F5008327C41766864E8582971C4883C50F
:10837000E4FF1389E4FFFD171CC88327C417668632
:108380004E858297CA840329040013790901631377
:10839000090C238004001C401307004093F707607A
:1083A000639EE7023386AB416396AB05D6850146F3
:1083B0004E85EF00F06218402A8AAE8A9376270035
:1083C00083270B00A9C6138747002320EB009C439B
:1083D00088C3CCC35C4485075CC4C1B9E3080AFC0C
:1083E0000146A94693051C004E85EF0070743306C4
:1083F0004541E2849307F41663E4F4009304E41621
:10840000974500009385C5602685D92045B793869A
:1084100047002320DB00118B844319CFAA855686A1
:108420000808EF309078D2466247F2474246D4C0FF
:1084300098C490C0DCC479BF2A86AE86EF30706DD8
:1084400009C50145412088C071B75285D685EFE046
:10845000DFD9D5BF014991B939713EDA2ED232D474
:1084600036D63AD842DC46DE9387C18022CC8043A0
:1084700026CA06CEAA8411C41C4C81E72285EF10BF
:10848000104D0C4454102686228536C6EF308034B9
:10849000F2406244D24421618280411122C42A8484
:1084A0002E8523A401CE06C6EFA06FFFFD576317EC
:1084B000F500938781CE9C4391C31CC0B2402244F7
:1084C0004101828097470000938707558843828047
:1084D00035713ECBB707008093C7F7FF3ECE3EC84D
:1084E000C1779387872032C536C73AC942CD46CF78
:1084F0003ECA9387C1802AC42ACC884334012E8681
:108500002C0086DE36C2EF20F07FA24723800700D2
:10851000F6500D618280AA87850703C7F7FF6DFFBC
:108520003385A7407D158280011122CC2A872E84B5
:108530003A85A28532C606CEEF20304032462A88E0
:10854000AE8805C651801374F47F9307B006818FFF
:10855000635DF000D2073707F03F01483E9742863F
:10856000BA86EFD05FDE2A88AE88F2406244428548
:10857000C6850561828035714AC92A89368532D41B
:1085800036C606CF22CD26CB4EC7EAD8EED62E8DE4
:1085900052C556C35AC1DEDEE2DCE6DA82C8EF20FD
:1085A0004046AA8D084181440144B537B246AA89A4
:1085B000EAC635469305B0021305D002130800023F
:1085C000A548B6479823636BE608637F170955C72C
:1085D00002C8364A93070003814A03470A00631B17
:1085E000F71283471A00130780056388E700130614
:1085F0008007130700036396C710C24736889808A0
:10860000D4081746000013066647EC004A85EF10B1
:10861000D05693797500AA8A6388090099476397B1
:10862000F906050AD2C602C8A25781C7B647225723
:108630001CC3C247B9C7B7050080A18DFA406A4480
:1086400026854A49DA44BA492A4A9A4A0A4BF65BCD
:10865000665CD65C465DB65D0D6182806309B700DD
:108660006303A702E31607F78507BEC699BF02C8D2
:1086700013871700BAC69C33A9FFA257EAC602C8DF
:10868000D5F7A28565BF05473AC8DDB7464611CA8A
:1086900093055003A808EF20704EC6454A85EF2089
:1086A000C045FD19914763EE3701174700001307D6
:1086B000E7368A09BA9983A70900BA978287E64400
:1086C000764493FA8A00E3810AF6B70700805D8C4E
:1086D000A1BFF6453704F0FF7D14B3F7850056447B
:1086E000E644130434439315440133E4B700D1BF87
:1086F0003704F07FF9B7B705008013C4F5FFFD54C8
:10870000C9B7B64793861700B6C69C33E38BE7FE1E
:1087100081DF854AB64C014A814B014CA546A145F3
:10872000A9473645034B050013070BFD1376F70FDA
:1087300063FDC60483A50D004E86EF30E03C3DC1CD
:10874000DA87E28D8146014B0145130750066387A6
:10875000E7001307500481496395E71663960D00FF
:10876000B3E7560199DB814D364D1307B0029307ED
:108770001D00BEC683471D00638FE70C1307D002A0
:1087800001486390E70E0548C1A863C98501B38B12
:10879000FB02BA9B0505050CAAC661B7330AFA02AB
:1087A0003A9ACDBF364581464E95AAC61C21630B29
:1087B0000C06014BE28D138707FD25466375E60223
:1087C000054561B7B647850613861700B2C69C33C8
:1087D000E38AE7FE1387F7FC2146E366E61EB64C04
:1087E000368B814D8146938707FD1387160085C719
:1087F0003A9B3385B6016E872148C14829466316E6
:10880000A702850DB69DA14663CEE6022947B38B2C
:10881000EB020147BE9BB64793861700B6C69C3352
:10882000BA8651BF1307000365B793051700634667
:10883000E800B38BCB022E87D9B7E3CEB8FE330A5C
:10884000CA02D5BFC1460147E3C7B6FDA946330AF0
:10885000DA023E9AC9B7014893072D00BEC6834786
:108860002D00138707FD25466365E60C13070003FB
:108870006385E70A1387F7FC214681496363E604B1
:10888000B648138707FD2543294EB64713861700C0
:10889000B2C69C33938507FD93F5F50F6375B30856
:1088A0009569330616419389F9E1A148CE8563C6DF
:1088B000C800BA8963D3E500AE8963040800B30930
:1088C000304163960D0CB3E6DA00E39F06D4E3165D
:1088D00005DA1307E0046389E706634FF70413071B
:1088E0009004E39CE7D89745000093852518E8009D
:1088F000EF101078E30305D8B6479745000093853D
:108900002517E800FD17BEC6EF10907601E5B647C3
:108910008507BEC63704F07F01BBB6471386170034
:10892000B2C69C33B1B73307C703BA97138707FDA5
:10893000A9BFEAC6814971B713079006E385E7FA34
:108940001307E006E39BE7D2974500009385C51225
:10895000E800EF10F071E30205D2B64798239307C1
:1089600080026313F702B008974500009385451213
:10897000E800EF10D07295476318F500F64537040C
:10898000F07FE6444D8C4DB13704F8FF71B9B38ADE
:10899000694163130C006E8CC1476E8D63D3B701C0
:1089A000414D5E85EFE0EFE6A547AA842E8463DCA7
:1089B000B70393077DFF139737009747000093870E
:1089C000E71EBA979043D443EFD0FF972A8452858D
:1089D000AE84EFE00FE42A86AE862285A685EFC03E
:1089E0005FC8AA842E84BD4763CDB709E38E0AC24F
:1089F000635450075947634357038E0A9747000053
:108A00009387C71ABE9A03A50A0083A54A00268643
:108A1000A286EFD05F93AA842E8439B11307500247
:108A20003307B741634F5705B38DB741174900006E
:108A30001309C91793973D00CA978843CC43B38D58
:108A4000BA412686A2868E0DEFD0FF8FCA9D03A65F
:108A50000D0083A64D0075BFA95763C4FA02B30980
:108A60003B41139B39009749000093892914DA99F7
:108A700003A6090083A649002685A285EFD06FB121
:108A800059BF338DAD41569D6357A0119377FD00BB
:108A900099CF17470000130767118E07BA978843CD
:108AA000CC432686A286EFD01F8AAA842E84137D0B
:108AB0000DFF63080D0A9307401363D5A705014B0B
:108AC000814902C6814B930720022320F900370415
:108AD000F07F8144B247E38907B4C6454A85EF2059
:108AE000C001DE854A85EF204001CE854A85EF2012
:108AF000C000B2454A85EF204000DA854A85EF1074
:108B0000D07F1DB6135D4D402685A2858147014A61
:108B10000548974800009388E8066346A80599C36E
:108B2000AA842E84174700001307C70593173A003D
:108B3000BA978843CC433707B0FC22972686BA867B
:108B4000EFD07F803704F07FB377B4003707A07C85
:108B5000AA84E366F7F63707907C637AF7027D1400
:108B6000FD54014ADDA813771D0011CF13173A00F9
:108B7000469710435443EFD00FFD8547054897486B
:108B8000000093882800050A135D1D4079B737045B
:108B900050032E94F9B7E3060DFC330DA0419377F3
:108BA000FD0099CF17470000130747008E07BA97BB
:108BB0009043D4432685A285EFD0AF9DAA842E840E
:108BC000135D4D40E30F0DF8FD4763DDA701014B39
:108BD000814902C6814B930720028144014423202E
:108BE000F900CDBD137A0D0163040A00130AA00633
:108BF0002685A285974700009387C7EA01479376A9
:108C00001D0081CA9043D4433EC6EFD0CFF3B24794
:108C10000547135D1D40A107E3130DFE19C3AA8488
:108C20002E8463050A029357440113F7F77F9307D5
:108C3000B006998F635CF0007D476354F7221307F9
:108C4000400381446359F72037047003014681468D
:108C50002685A285EF30004F3DD95E87EE8662867D
:108C6000E6854A85EF1030772AC6E30A05E493D7F4
:108C7000FA41B3093B41B3F7F9003ED056CE63D376
:108C80000A0002CEB247014B8149B1073ED8B7076F
:108C90001000FD173ED6B2474A85CC43EF10305D39
:108CA000AA8BE30205E2B247C2553105904B090693
:108CB0000A06EFE04FF2B808D4082286A6854A8556
:108CC00026CA22CCEF200057AAC8E30E05DE854550
:108CD0004A85EF208005AA89E30705DED64763C7EA
:108CE00007180257724C338DE7006647B387474138
:108CF00093066003BA97FD17930D20C0998E63D633
:108D0000B7193387FD407D46998E6346E616854D3B
:108D1000B397ED003ED2814C369CB30DDD00529CE2
:108D2000EA8763D3AD01EE876353FC00E2876358A3
:108D3000F000B38DFD40330CFC40330DFD408257F5
:108D40006358F002CE853E864A85EF200014AA893A
:108D5000E30B05D64646AA854A85EF10D07E2ADA6F
:108D6000E30305D6C6454A85EF103059D257BEC831
:108D7000634FB011635A50017246DE854A85EF2079
:108D8000C010AA8BE30105D4635A8001DE85628698
:108D90004A85EF20601BAA8BE30705D2635AA00126
:108DA000CE856A864A85EF20201AAA89E30D05D070
:108DB000C6455E864A85EF2020292A8BE30505D02B
:108DC000032CC500CE8523260500EF20C02463595F
:108DD000050C336C9C0063110C129317C400639D47
:108DE0000710B707F07FE18F3707B0066376F710FB
:108DF00083274B0191E703270B01854763DEE70ECD
:108E0000DA8505464A85EF202014CE852A8BEF208F
:108E100080206353A00E630C0A10B707F07FE18F28
:108E20003707B0066345F71037077003E355F7DAE5
:108E30000147B70750392685A2853A86BE86EFD00E
:108E40008FD02E84C98DAA84E39905C89307200288
:108E50002320F90059B181177D57B317F7007D8C96
:108E6000F5B37D57B317F700FD8CCDB37247025DA4
:108E7000330CF7409DBD930C20BEB387FC40854C5E
:108E8000B39CFC0085473ED241BD814CE5BFC64541
:108E90006E864A85EF20400BAAC8E31D05EC25B17C
:108EA00069E9370710007D17B377E40063090C0404
:108EB0006399E7047D5763000A02B707F07FE18FEB
:108EC000B706A00663E9F600D1839306B006B38720
:108ED000F6403317F7006396E402B707F07FFD17FB
:108EE0006315F400FD57E380F4BEB705F07FE18D14
:108EF000370410002E948144E31C0AF2F9BEC58F9A
:108F000099DB63820C04B3FC8C00E3870CFE528671
:108F10002685A285630F0C02EFF00FE12A86AE864C
:108F20005245E245EFC0EFF3AA842E84F1B7B705AE
:108F3000F07FE18D3704F0FFA295370410007D1417
:108F40004D8CFD5455BF9257B3FD9700E3860DFA43
:108F50007DBFEFF06FDD2A86AE865245E245EFD049
:108F60001F8A01468146AA842E84EF30A01D49F550
:108F70009DB1CE855A85EF20203997470000938711
:108F800067AC9043D4432A8DAE8DEF30202D6342E1
:108F9000A01063010C0A814D370DF03F0147B70760
:108FA000F03FB706F07FB37CD400B706E07F639F45
:108FB000DC166AD2370DB0FC229D2685EA853EDE9E
:108FC0003ADC6EDAEF206017D25812582A86AE8645
:108FD0004685C285EFD02FB72686EA86EFC06FE8B8
:108FE000AA843705F07F3376B500B706A07C6257B8
:108FF000F2576365D60C62479307F5FF6396E70067
:109000005247FD57E381E7ACB707F07F1384F7FFC2
:10901000FD54C6454A85EF10502EDE854A85EF1077
:10902000D02DCE854A85EF10502DDA854A85EF1078
:10903000D02C95B1B1E0B257E18FA1E7974700007E
:109040009387C79F9043D4436A85EE85EF30002114
:10905000634D0502974700009387C79D9043D44313
:109060006A85EE85EFD02FAE2A87AE87370D008058
:10907000BA8D334DFD0035B785476394F400E30C9A
:1090800004B4814D370DF0BF11BF0147B707E03F72
:10909000F1BF974700009387E7999043D4436A85CF
:1090A000EE85EFD04FAA2A87AE872E8D63160C006F
:1090B000370D0080334DBD00AA8DE5B53704500350
:1090C0002E94E3180AF4B706F07FE18EE393DCF404
:1090D000BE853A853A8DBE8CEFD03FE6EFD07FEC6F
:1090E0002A86AE866A85E685EFD06FF1B2572A8D63
:1090F000AE8DE18FC58F33EC8701630B0C0A974768
:109100000000938727959043D443EF302015E34622
:10911000059C97470000938767949043D4436A85E2
:10912000EE85EF30C008E356A0EE45BA630D0A04A1
:10913000B706A00663E99605974600009386069158
:109140009042D4423A85BE853ADA3ED2EF300011E1
:10915000925752576344A0023A85BE85EF30201FD4
:1091600011E10545EFD0FFEA2A87AE872E8D631601
:109170000C00370D0080334DBD00AA8DB705B00639
:109180002E9D330D9D415245E2453EDA3AD2EF1015
:10919000D07A2A86AE866E85EA85EFD0CF9A52467F
:1091A000E246EFC00FCCAA842E84D257125711BFCB
:1091B000974700009387078B9043D443EF30000A12
:1091C000E35905E419BA130750066387E70013074C
:1091D000500405456399E7EE014B05456FF04FD804
:1091E0009387C1809C43945389E69776FF1F9386AB
:1091F00066E86FF04FB879714AD04ECE06D622D4C9
:1092000026D2AA892E899304190003C4F4FF3A8553
:1092100036C632C42EC23AC0EF10407E22951C31B1
:1092200002479245A18B2246B246D1E39307D00272
:109230006311F4089C20054393042900E5C64147C7
:109240006390E60213070003639CE7009C2013076A
:10925000800593F7F70D6392E70C9C30C1468904B3
:10926000B70800806314030093C8F8FF33FFD802E7
:1092700001480145A54FE54EFD5233DED802138764
:1092800007FD63E3EF04BA8763DED704630D58007C
:109290007D58636AAE006314AE006346FF00054864
:1092A0003385A6023E95850483C7F4FFC9BF26898E
:1092B00099BF9307B0026305F400A2870143BDBFC5
:1092C0009C2093042900DDBF1387F7FB63E5EE00C4
:1092D000938797FC55BF1387F7F963E5EE009387F3
:1092E00097FA5DB7FD57631FF8009307200223A08C
:1092F000F900468519EEB250225492540259F249AF
:1093000045618280630403003305A0406DD6630489
:1093100008009385F4FF0CC2F9BF93070003A9F27C
:10932000A1463DBF13070003E382E7F2A9460DBF44
:109330009387C1809C43985309E71777FF1F130752
:1093400067D36FF05FEB011122CC1C49804906CE38
:1093500026CA4AC84EC652C456C263C187127D147B
:109360001318240093894501338A09011309450123
:109370004A9883270A00032708008507B354F70299
:109380006366F706C1684E834A8E814E014FFD1811
:1093900011030326C3FF110E3377160141823307F1
:1093A000970233069602769793560701B377170113
:1093B000B307FF4036968326CEFF935E06013376D1
:1093C000160133F71601BA97C18213D70741918E60
:1093D000BA9613DF0641B3F71701C206D58F232EC5
:1093E000FEFEE3776AFA83270800BDCBAA8AEF1056
:1093F00090426349050441668504CA8501457D168E
:10940000910903A8C9FF98419105B376C800158D4D
:10941000B376C700AA96935707011358080113D7CC
:109420000641B3870741BA9713D50741F18EC207AA
:10943000D58F23AEF5FEE3753AFD93172400CA9746
:1094400098431DC72685F2406244D2444249B2493E
:10945000224A924A056182808327080089E77D14A9
:109460007118E36B09FF00C951B7984309E77D14F0
:10947000F117E36CF9FE23A88A00E9B70145E1B7CB
:1094800075713ED85C5122C526C34AC1CEDED2DCFE
:10949000E2D406C7D6DADAD8DED6E6D2EAD0EECE05
:1094A00036C23AC646CAAA842E843289C2892E8A16
:1094B000328C89EF4145EFD0DFF0C8D02322050080
:1094C000232405002320050023260500DC508C43BF
:1094D00089CDD84385472685B397E7009CC5D8C179
:1094E000EF10A061DC5023A00700635309048547F7
:1094F000131C190023A0F900135C1C00B707F07FB0
:109500003377FC006314F70642578967320C938760
:10951000F770135CCC001CC3336C8C00E3000C327E
:10952000D24791EB973700009387875E3EC039A8FA
:1095300023A00900E1B7973700009387675D3EC01D
:10954000973700009387F75C52471CC3BA402A4400
:1095500002459A440A49F659665AD65A465BB65BA2
:10956000265C965C065DF64D496182800146814627
:109570002285E28522CE62D4EF20D03C05E142571D
:1095800085471CC3973700009387C7453EC0D24725
:10959000D5DF973700009387F7447DB7B800F40014
:1095A0006286A285268513594C01EF10B0481379C5
:1095B000F97FAA89A64A630D0910A25772451309BB
:1095C00019C09395C700B181B707F03FDD8D02DC6C
:1095D000973700009387874F9043D443EFD02FA253
:1095E000973700009387074F9043D443EFC0BFD510
:1095F000973700009387874E9043D443EFC06F8620
:109600002A8B4A85AE8BEFD0DF999737000093877E
:10961000674D9043D443EFC01FD32A86AE865A8548
:10962000DE85EFC00F842A8BAE8BEFD01F912A848A
:10963000014681465A85DE85EF205042635B050076
:109640002285EFD01F965A86DE86EF20B02F11C1FB
:109650007D140547D9473AD663E3870213173400D0
:109660009737000093878754BA979043D443724545
:10967000A255EF20B03E635305007D1402D6338916
:109680002A41930BF9FF014B63D60B00054B330BBB
:109690002B41814B634E0406A29B22CC814A124788
:1096A000A54763E5E7149547854C63D6E700930724
:1096B000C7FF3EC2814C12478D47630EF71063CF40
:1096C000E704894702C8630DF70685473EC88DA0A9
:1096D00036499307000256991307294363D5E702D9
:1096E00013050004198D930729413315AC00335439
:1096F000F400418DEFD0FF91B70710FEBE9585476E
:109700007D193EDCF1B53385E7403315A400DDB7A4
:10971000330B8B40B30A804002CC51B712479147BC
:10972000630EF70005473AC8124795476306F70AE4
:10973000FD573EC4FD5DC94702C619A885473EC80E
:10974000B2476348F00A854705473EC4854D3AC68F
:1097500003A94402114723220900930647018325E8
:10976000490063FCD7082685EF106030DC502320C9
:10977000A9009C433EC0B94763E6B71D63840C1C37
:10978000635E800A9377F40013973700935C44403C
:109790009737000093878741BA9793F60C01984357
:1097A0000949DC4385C6973600009386A63D905252
:1097B0007245D452A2553AD03ED2EFC08FDD025747
:1097C000925793FCFC002A8A2E8C0D49173D00000D
:1097D000130D4D3B89A802C8B247A2973EC4938D92
:1097E0001700EE87E346B0F785479DB7854C02C268
:1097F000E9BDB2473EC4BE8DA1BF85052322B90095
:109800000607A1BF93F61C0081CE03260D00832618
:109810004D003A85BE85EFC01FB305092A87AE8784
:1098200093DC1C40210DE39F0CFC3A86BE865285DA
:10983000E285EFC00FD62A8A2E8C81A0094915CC6B
:10984000B30C804093F7FC00139737009737000064
:109850009387C735BA979043D4437245A25593DC9A
:109860004C40173D0000130DED31EFC0DFAD2A8AEB
:109870002E8C8147639B0C12DDFFB2576386071461
:10988000173700001307871B104354435285E285A6
:1098900052D0EF20B01C63590512638A0D12A24703
:1098A0006350F00A1737000013074724825710430C
:1098B00054433E85E285EFC01FA9A247130DF4FF74
:1098C0002A8A2E8C050962874A853EDE52DABA8CD6
:1098D0003AD0EFD00FED525802573709C0FC4286FC
:1098E000BA86EFC05FA6973600009386A620904206
:1098F000D442528CEFB0FFD6F2572A8A2E99F9EB58
:10990000973700009387871F525802579043D443DC
:109910004285BA85EFC0BFEE5286CA862A8CAE8CCD
:10992000EF20F0086346A054B7070080B3C72701B3
:109930005286BE866285E685EF2050126347055247
:10994000724A225CB64763C30730394763408730A9
:10995000131734009737000093874725BA9703AB56
:10996000070083AB4700B24763D10720634FB01FA6
:10997000639D0D4E97370000938747189043D4435B
:109980005A85DE85EFC03F9C5286E286EF2030028A
:10999000814A01496353054A824702470504138AF5
:1099A0001700930710031CA369A913F71C0009CB28
:1099B00003260D0083264D000509EFC0DF9885477B
:1099C00093DC1C40210D7DB5228DEE87EDBD228DEF
:1099D0008147D5BD9386F7FF139636009736000072
:1099E0009386C61CB2968842CC428246B6973EDA2F
:1099F000C247E9C3973700009387C7032A86AE861C
:109A00008843CC434ADE52D0EFC0AFB802587257F9
:109A1000173900001309890D4286BA86EFC03FDE70
:109A2000024A2AD02ED2E6856285EFD00FD12ADEF7
:109A3000EFD02FD72A86AE866285E685EFC03FDC61
:109A4000F2572A8CAE8C2A86AE8602559255050AAC
:109A500093870703A30FFAFEEF2060756348A00EFB
:109A600097370000938787FD8843CC436286E6865C
:109A7000EFC0FFD82A86AE8602559255EF2020739C
:109A80006342A018D257E30DFAEA032609008326A1
:109A9000490002559255EFC01F8B0326090083260B
:109AA00049002AD02ED26285E685EFC0DF892A8C54
:109AB000AE8C95BF5286CA86EFC0FF88525A0249C3
:109AC0002AD02ED2E6856285EFD02FC72ADEEFD0CE
:109AD0004FCD2A86AE866285E685EFC05FD272578B
:109AE000D257050913070703A30FE9FE2A8CAE8C92
:109AF0006312F906173900001309C9F30326090098
:109B00008326490002559255EFB0BFB52A86AE862E
:109B10006285E685EF20A0696346A00E0256925644
:109B20000325090083254900EFC07FCD2A86AE8634
:109B30006285E685EF20807293070003E35205E01B
:109B40000347FAFF9306FAFF6304F7006A8459A8F3
:109B5000368AFDB797370000938747F99043D4437F
:109B6000EFC06FFE2A8CAE8CB1BFE287BE8C8247FD
:109B7000528C973A0000938A6AF713891700BE9DAA
:109B80005A86DE866285E685EFC0AFA0EFD0EFBAD9
:109B90002A8DEFD00FC15A86DE86EFC0CFFA2A8613
:109BA000AE866285E685EFC09FC593070D03A30FC0
:109BB000F9FE2A86AE864A8A639B2D07EFB07FAAFC
:109BC0005A86DE862A8CAE8CEF20605E634BA00244
:109BD0005A86DE866285E685EF20C05601E59377DA
:109BE0001D0085E3CE852685EF003071C257230026
:109BF0000A00050480C3D247E38A079423A04701E3
:109C0000B1B2228D130790038346FAFF9307FAFF40
:109C10006399E6008246639AF60013070003050D78
:109C200098A29823050798A315B73E8AF1BF03A60B
:109C30000A0083A64A000509EFC0EFF001468146FD
:109C40002A8CAE8CEF20005005FD69BF42476300AF
:109C50000710924605476345D70C625793873743F1
:109C600009E7264793076003998F568DDA8C85455F
:109C700026853E9BBE9BEF10400B2A89635E9001B8
:109C8000635C7001E68763D39B01DE87330BFB4087
:109C9000B38CFC40B38BFB4063800A04C247C5CF42
:109CA0006354A003CA856A862685EF10001E4E867F
:109CB000AA852A892685EF1000092ACECE85268519
:109CC000EF00B063F247BE893386AA4111C6CE8544
:109CD0002685EF10801BAA8985452685EF10E004B4
:109CE000E247AA8A635BF0063E86AA852685EF10C6
:109CF000C01912478547AA8A014D63C8E706014D7E
:109D000063120A069317CC00528DA9EFB705F07FB6
:109D1000337CBC0063080C04050B850B054D99A032
:109D2000138DFDFF63CAAA01338DAA4163DE0D00C6
:109D3000B30CBB41814725BFE247B30A5D41D697CB
:109D40003ECCEA8A014DDDB7DA8CEE870DB7568D31
:109D5000DA8C014925B756869DBF12478547014DCC
:109D6000E3DFE7F8E247054589CF83A70A018D07BE
:109D70008A07D697C843EF005070930700023385D7
:109D8000A7405E957D8951C193070002898F1147D5
:109D9000635AF706F1473385A7402A9BAA9CAA9BE2
:109DA00063586001CE855A862685EF10E019AA898E
:109DB00063587001D6855E862685EF10E018AA8A62
:109DC000B257B1C7D6854E85EF10E0246351050424
:109DD000CE85814629462685EF007056C2477D1400
:109DE000AA89638B0726CA85814629462685EF0006
:109DF0001055A2472A896345F0081247894763D165
:109E0000E70829A8E38EE7F83E85710579B7634531
:109E1000B0071247894763D1E7066EC4A24791EFA6
:109E2000D685814615462685EF007051AA8AAA85F7
:109E30004E85EF10401EE341A0B6B247024A13C45C
:109E4000F7FF014BD6852685EF00304BE30C09D890
:109E500063080B0063062B01DA852685EF00F049C5
:109E6000CA852685EF007049B5BB814A0149F1B723
:109E70006A84814A01490DB6C2476EC46385071ED4
:109E800063589001CA8566862685EF10E00B2A8903
:109E90004A8563060D02832549002685EF00303D83
:109EA000032609012A8B9305C90009060A06310514
:109EB000EFD06FD20546DA852685EF10E00882479D
:109EC00022474A8B138C1700BA973EC693771A0025
:109ED0002A893EC4D6854E85EFF0EFC6DA852A8DF5
:109EE000930D05034E85EF1000134A86AA8BD68585
:109EF0002685EF1060155045930CFCFF2A8A054714
:109F000011E6AA854E85EF1000112A87D285268595
:109F10003AC8EF00903E92474247628AB3E6E700B4
:109F2000A247DD8E81EE130790036388ED0463542E
:109F30007001930D1D032380BC0129B763CA0B0078
:109F40009247B3EB7701A247B3EBFB0063950B0499
:109F5000E353E0FECE8505462685EF00F07ED685EC
:109F6000AA89EF10400B6346A00071F513F71D009E
:109F700079D313079003E39EEDFA930790032380B0
:109F8000FC00930690038347FAFF1307FAFF638CE4
:109F9000D708850745A0635BE00013079003E38EB5
:109FA000EDFC93871D002380FC0069BDB247A30F21
:109FB000BCFF63818705CE85814629462685EF0053
:109FC0001038AA8981462946DA85268563182B012F
:109FD000EF00F0362A8B2A89050CEDBDEF003036F4
:109FE000CA852A8B814629462685EF0050352A8965
:109FF000E5B7014BCE8505462685EF00F074D68582
:10A00000AA89EF104001E34EA0F601E593F71D0089
:10A01000ADFB930700030347FAFF9306FAFFE31330
:10A02000F7E2368ACDBF82476398E700024705040E
:10A03000930710031CA339B53A8AB1B75247973733
:10A040000000938727AC3EC097370000938707AC8A
:10A05000631C07CE6FF08FCFA2476346F000124714
:10A060008947E3CDE7DA024AD6854E85EFF0AFADFA
:10A070008247050A930D05033307FA40A247A30F51
:10A08000BAFFE358F7F6CE85814629462685EF00CC
:10A09000102BAA89D1BF411122C406C62A844EA51D
:10A0A00072A5232005002322050023240500232276
:10A0B000050623280500232A0500232C0500214638
:10A0C00081451305C505EF60AF8B97270000938787
:10A0D00047995CD0972700009387679B1CD49727EC
:10A0E00000009387479F5CD4972700009387A7A120
:10A0F00000D01CD8B2402244410182809725000044
:10A100009385A5D999AA411126C213068006938486
:10A11000F5FFB384C4024AC02E8922C406C69385C3
:10A120004407EFD0EFC02A8401CD2320050023226D
:10A130002501310508C4138684068145EF604F84EC
:10A140002285B240224492440249410182801C4D42
:10A15000A5E7411106C622C497070000938747FA76
:10A160001CD5938701819C432324050423260504E1
:10A17000232805046314F50085471CCD2A8435285F
:10A1800048C022851D2808C42285052848C44840A7
:10A1900001469145EFF03FF008440546A545EFF034
:10A1A0009FEF48440946C945EFF0FFEE85471CCCB8
:10A1B000B240224441018280828041119387018113
:10A1C00026C284434AC006C69C4C22C42A8981E721
:10A1D0002685EFF0DFF7938484048044DC40FD178C
:10A1E00063D607009C40B9CF8440C5BF0317C400A5
:10A1F00039E7C177850723220406232004002322A0
:10A200000400232404005CC423280400232A04003F
:10A21000232C0400214681451305C405EF505FF649
:10A22000232A0402232C04022324040423260404E6
:10A230002285B240224492440249410182801304A3
:10A24000840671BF91454A85EFF0FFEB88C049FD58
:10A25000B1472320F9000144E1BF797122D44AD0EB
:10A2600052CC56CA5AC85EC606D626D24ECE2A8AC6
:10A27000AE8A130485040149054BFD5B09ECB2501D
:10A2800022544A8592540259F249624AD24A424BB8
:10A29000B24B45618280044483294400FD1963D494
:10A2A00009000040E1BFDE24637BFB008397E400EC
:10A2B00063877701A6855285829A3369A9009384C2
:10A2C0008406E9BF10499306450113D75540B68768
:10A2D0006356C7020A060A07FD8936963697B9C93A
:10A2E000130847001843130300023303B3403357E6
:10A2F000B700636EC80098C311C391073387D74076
:10A30000098718C96394D700232A0500828083280F
:10A31000080091071108B398680033E7E80023AEFE
:10A32000E7FE0327C8FFE1B711078325C7FF9107A1
:10A3300023AEB7FEE36AC7FED1B7930705FD93F7D7
:10A34000F70F25476367F70001159377F50F3E85F3
:10A3500082809307F5F993F7F70F954663E5F600CA
:10A36000130595FBDDB71307F5FB1377F70F81474F
:10A37000E3EFE6FC130595FDC9BF1D71D6C2AA8A9D
:10A38000428536C63AC286CECAC8D2C4DAC05EDEBC
:10A390003E8B6ED63289AE8DA2CCA6CACEC662DC0A
:10A3A00066DA6AD8B92D832B05005E85EFE0AF969B
:10A3B000B387AB0083A60D0083C7F7FF7957158FCE
:10A3C0003EC82A8A93872600930600033306F700C7
:10A3D000BE84850703C5F7FF32C4E309D5FEEFF05D
:10A3E000DFF5631E05105286DE852685EF10C071ED
:10A3F000631C0510338C440103450C00EFF0FFF3A0
:10A4000063050510E284930700038820630BF500C1
:10A41000EFF0BFF2854793391500E28C3EC4268CDD
:10A4200021A08504DDB7050C03450C00EFF0FFF01B
:10A430007DF95286DE856285EF10006D11E9639C1F
:10A440000C00529CE28C03450C00EFF01FEF5DE91D
:10A45000014463850C0033848C410A0483470C005B
:10A46000130700056387E70013060007E28C63907B
:10A47000C70683471C001307B002638BE708130766
:10A48000D002638BE708930C1C00014D03C50C0040
:10A49000EFF0BFEA9307F5FF93F7F70FE14563E4A9
:10A4A000F508930705FF850C03C50C003ECAEFF0C5
:10A4B000DFE89305F5FF93F5F50F6148D247A9480A
:10A4C000637EB80463040D00B307F0403E9423A0FC
:10A4D0009D01638C0904A247814491E39944F640AD
:10A4E000664426854649D644B649264A964A064BCE
:10A4F000F25B625CD25C425DB25D25618280814923
:10A50000814C31BF050C81B7268C01448549B9B710
:10A51000014D930C2C009DBF054DE5BFB38717037C
:10A52000AA97C11749B7E28C5DB7B3079C40FD17E6
:10A5300081451D476343F70A5685152B0546930948
:10A540004501B3074641AA8D4E8D8148814C3ECAD4
:10A5500063E8840913054D0033053541098523203F
:10A560009D0123A8AD009314550066853927832BE0
:10A570000900898C63D89B0CB3847441A6856E85D1
:10A58000EF0030632A8A05C91386F4FF93565640BC
:10A590008A06CE96944205473317C700758F054A41
:10A5A00019CB6359CA009385E4FF6E85EF00706094
:10A5B0000D4A11E1094AA6856E85EFF0BFD02694B9
:10A5C00003278900635F8708EE8556853D23924700
:10A5D0009304300A23A0070019B78505858799BF22
:10A5E0009307FCFF3EC40346FCFFC2476309F60223
:10A5F000930700026397F80023209D018148110D05
:10A60000814C0345FCFF46CCEFF03FD3E2483D8947
:10A61000224333151501B3ECAC00910815A0524745
:10A620009307FCFF3383E700E36493FC1A855286AB
:10A63000DE8546CE1ACCEF10204D6243F2484DF92C
:10A640001A8C39B7014AE3DD74F7B3849B40EE8579
:10A6500026865685EF00500FAA8D058C930945017B
:10A6600085B7032749006355E40E330487406345EB
:10A6700074070327C9008946630AD7048D46630A15
:10A68000D7048546631BD70263998B026391EB0263
:10A6900003274900B2479304200698C30547924711
:10A6A00023A8ED0023A0E90023A0B7010DBD9385E9
:10A6B000FBFF6E85EF00F04F61FDEE855685352975
:10A6C00092479304000523A0070011BDE3170BFE7A
:10A6D000C1B7E31F0BFAD5B79304F4FF63180A065A
:10A6E00091C4A6856E85EF00D04C2A8A13D75440BA
:10A6F0000A074E9718438545B3959500F98D99C182
:10A70000136A2A00A2856E85B38B8B40EFF09FBB46
:10A71000032449008944630B0A080327C9008946BA
:10A72000630AD7028D46630AD7028546631DD700A8
:10A7300013772A0009CB03A70900336AEA00137ACA
:10A740001A00631E0A0093E404018DA0054A79BF34
:10A750008544D1B70547330B6741E3060BFE83A958
:10A760000D0113874D01FD55139A2900330647014A
:10A7700014436383B604850614C3894613874D01C9
:10A780006394D40883260900FD16639F760193D64F
:10A790005B408A06369718438546B39B7601B3FB28
:10A7A000EB0063830B00854493E40402924723A0EB
:10A7B000B701B24780C325B31107232E07FEE36913
:10A7C000C7FA03A78D0063C5E90283A54D0056852E
:10A7D0008505712C03A60D019385CD002A8B0906F2
:10A7E0000A063105EFC03FBFEE8556853926DA8D62
:10A7F00003A70D019306170011070A0723A8DD0020
:10A800006E97854654C395BF83A60D0163DCD900BE
:10A8100085456E85EFF01FAB032789000504E354DF
:10A8200087F85DB393FBFB018544E38F0BF65297EA
:10A830000325C7FF992113070002B30B7741E349B2
:10A8400075FD9DB7A1473386C7400A0693060002EF
:10A85000918E5C41184111053398D7003367070189
:10A86000B3D7C700232EE5FE1CC1E364B5FE82808A
:10A870001C416548850503C6F5FF850701E61CC137
:10A880000545828098239306F7FB93F6F60F6364E1
:10A89000D80013070702E30FC7FC014582805D71F2
:10A8A00052DC03AA0500A6C24EDE93545A405AD881
:10A8B0008A0486C6A2C4CAC056DA5ED662D466D2FC
:10A8C0006AD06ECE137AFA012A8BB289B2946303EE
:10A8D0000A00910483270B001389C4FF23AE04FEF2
:10A8E000CA8D4A840146814A814B214C930C000257
:10A8F0001D4D9433138717003AC0B1CA368532C64E
:10A900003EC436C2EFF07FA3324659E59246A247D5
:10A9100063E8DC0263D47A036378B4016346CD0054
:10A92000EE852285EFF01FF2214663F98900930D31
:10A93000C4FF232E04FEDE8A6E840146824755BF83
:10A9400093059002639CB60889072320FB00638768
:10A950000B086379B4019D4763C6C700EE85228565
:10A96000EFF05FEE63FA8904CE8711040327C4FF7A
:10A97000910723AEE7FEE37A89FE910723AE07FE37
:10A98000E37DF9FE8327090091E7631739058547C1
:10A990002320F9001545A1A00506850B6358CC00BE
:10A9A000E3FE89F8232E04FE054671141C403D8900
:10A9B0009207C98F1CC059B7E3060AFC930700022F
:10A9C000B38747417D5AB357FA0003AAC4FF337ACD
:10A9D000FA0023AE44FF7DB771196DB71145B6403B
:10A9E000264496440649F259625AD25A425BB25BF7
:10A9F000225C925C025DF24D616182800325C50E8E
:10AA000082801305050F82809387C1809C43885301
:10AA100009E51755FF1F1305E5651305050F82802E
:10AA200091ED41116C00014501CA795591C61C2276
:10AA30009CC108223335A00041018280014509CA2A
:10AA4000795599C61C229CC108223335A00082800A
:10AA5000828093F5F50F2A966314C5000145828024
:10AA60001C21E38EB7FE0505C5BF828082805C5144
:10AA7000411122C44AC006C626C22A842E8989EF03
:10AA80004145EFC01F9448D0232205002324050030
:10AA900023200500232605004450DC449DC7585060
:10AAA000931729005847BA97884329E18544B394FE
:10AAB0002401138654000A0685452285EF00D01331
:10AAC00019CD2322250104C525A0130610029145A6
:10AAD0002285EF0070125C50C8C4DC47E9F30145E1
:10AAE000B24022449244024941018280184198C3F5
:10AAF0002328050023260500E5B75C51011122CC6F
:10AB000006CE2A8499EF41452EC6EFC09F8BB245F1
:10AB100048D02322050023240500232005002326F6
:10AB2000050091C95450DC4113972700DC46BA97C1
:10AB3000984398C18CC3F240624405618280797168
:10AB40004ECEAA89416522D426D22E84844906D6C7
:10AB50004AD0D10501487D159C419105050833F780
:10AB6000A7003307C702C183B387C702369793563E
:10AB70000701698FB69793D60701C207BA9723AE2C
:10AB8000F5FEE34B98FCA1C21C4463C7F4024C40A1
:10AB90004E8536C68505EFF09FED10489305C4003D
:10ABA0002A8909060A063105EFC0FF82A2854E8573
:10ABB000EFF0BFF4B2464A84938744008A07A29715
:10ABC000D4C3850404C82285B25022549254025939
:10ABD000F2494561828079719387860052CC368A2A
:10ABE000A54622D426D24ECE2E84B3C7D70206D68F
:10ABF0004AD056CAAA89B2848546814563CCF604F8
:10AC00004E853AC6EFF0BFE6324785471CC958C9A2
:10AC1000A54763D49704930A94005689269405099E
:10AC20008346F9FFAA852946938606FD4E85EFF0F7
:10AC30001FF1E31689FE138484FF5694268963412D
:10AC40004903B250225492540259F249624AD24AFC
:10AC5000456182808606850555B72904A544F9BF5C
:10AC6000B3079940A2979423AA852946938606FDA7
:10AC70004E85EFF0DFEC0509D9B74177698FAA87D8
:10AC8000014519E3C2074145370700FF7D8F19E3EE
:10AC90002105A207370700F07D8F19E31105920700
:10ACA000370700C07D8F19E309058A0763C90700CC
:10ACB00013971700050563440700130500028280FF
:10ACC0001C4113F777000DC393F61700014799E66F
:10ACD00013F7270011C785831CC105473A85828079
:10ACE00089831CC10947DDBF93960701C1820147D3
:10ACF00099E2C183414793F6F70F99E22107A183B7
:10AD000093F6F70099E21107918393F6370099E2E1
:10AD10000907898393F6170081E68583050799C3A0
:10AD20001CC16DBF1307000255BF411122C42E8400
:10AD3000854506C6EFF0BFD340C9B240224405475F
:10AD400018C94101828098491C4A797126D206D6D9
:10AD500022D44AD04ECEAE846354F700B2842E86FD
:10AD600083A90401032906019C44CC4033842901B2
:10AD700063D38700850532C6EFF07FCF32461308D4
:10AD80004501131324004293C28763ED6702938544
:10AD90004401939829005106131E2900C166AE98FC
:10ADA000329EFD166364C6036356800071138327C9
:10ADB0000300F1CB00C9B250225492540259F24917
:10ADC0004561828023A007009107C1B7832F060049
:10ADD000B3FFDF00638A0F04428FAE82814403A772
:10ADE000020083230F00110FB37ED700B38EFE0342
:10ADF000B3F7D30093D303019102BE9E935707018B
:10AE0000B387F703A69E13D70E01B3FEDE009E970D
:10AE1000BA9793D40701C207B3E7D701232EFFFEE9
:10AE2000E3EF12FB23209F0083522600638A020473
:10AE300083270800C28E2E8F814F03270F0083D3F4
:10AE40002E00F58F758F33075702910E110F1E9745
:10AE50007E97931F0701B3E7FF0023AEFEFE8357E3
:10AE6000EFFF83AF0E004183B3875702B3FFDF00CC
:10AE7000FE97BA9793DF0701E3611FFD23A0FE0051
:10AE80001106110805B77D1405B7011126CA4AC875
:10AE90004EC606CE22CC52C4937736002A89B2849D
:10AEA000AE8989CFFD17172700001307A7DC8A0793
:10AEB000BA9790438146EFF09FC8AA898984A5CCB0
:10AEC0008327490291EF4145EFC0AFCF2322A9026A
:10AED0002322050023240500232005002326050046
:10AEE000032A490203248A0019E8930510274A859A
:10AEF000EFF0BFE32324AA002A842320050093F760
:10AF0000140081CFCE8522864A85EFF0DFE32A8ABE
:10AF1000CE854A85EFF07FBED289858489CC0840F2
:10AF200009E92286A2854A85EFF0FFE108C02320C7
:10AF300005002A84E9B7F24062444E85D244424972
:10AF4000B249224A05618280797126D2AE844ECE02
:10AF500083A9040122D4CC41135456409C44A299A5
:10AF60004AD056CA06D652CCAA8A1389190063C49D
:10AF70002709568532C6EFF09FAF32469307450149
:10AF80002A8ABE8601479106634A870663530400F6
:10AF9000014494480A04338787008A069387440152
:10AFA0007D8ABE9625C2130800023308C840814539
:10AFB0008843110791073315C500C98D232EB7FEAD
:10AFC00083A5C7FFB3D50501E3E4D7FE0CC399C140
:10AFD000138929007D1923282A015685A685EFF0BB
:10AFE000DFB1B2502254528592540259F249624A5A
:10AFF000D24A456182808505860795BF23AE06FE4D
:10B00000050751B7910703A6C7FF1107232EC7FEF7
:10B01000E3EAD7FEC1B71C499849998F8DE30A0727
:10B020005105D105B306E500BA95F116F115904228
:10B0300098416308E600FD576363E60085473E8557
:10B040008280E364D5FEE5BF011126CAAE844EC6F8
:10B05000B285AA89268522CC06CE4AC83284EFF072
:10B060009FFB05E181454E85EFF07FA085471CC918
:10B07000232A0500F2406244D2444249B2490561A4
:10B080008280054963460500A28701492684BE8463
:10B090004C404E85EFF0BF9D0323040183A80401BB
:10B0A00013064401131E2300138844018A08C16E4D
:10B0B00023262501329EC29893064501014FFD1EAD
:10B0C0001842832F08009106B375D701B3F7DF014B
:10B0D000FA959D8D93DF0F0193570701B387F741D1
:10B0E00013D70541BA9713DF0741B3F5D501C2075E
:10B0F000CD8F110823AEF6FE1106E36318FDC1657E
:10B10000FD156368C601F1169C4295C723286500AA
:10B1100095B71C429106110633F7B7007A9713587A
:10B120000741C183C29713DF07416D8FC207D98FD3
:10B1300023AEF6FEF9B77D13F9B7B707F07FFD8DA3
:10B14000B707C0FCBE956355B00081473E8582803D
:10B15000B305B04093D745414D476347F700B70566
:10B160000800B3D5F540D5B71387C7FEF94681452A
:10B170008547E3CDE6FCB7070080B3D7E700F9B712
:10B18000797126D204494ECE930945018A04CE94A2
:10B1900022D403A4C4FF4AD02EC6228506D6EFF0DF
:10B1A000DFADB24593070002898F9CC1A94713897F
:10B1B000C4FF63CDA702AD47898F3707F03FB35671
:10B1C000F400D98E014763F4290103A784FF5505D4
:10B1D0003315A400B357F700C98FB25022549254CC
:10B1E0000259F2493E85B68545618280814763F602
:10B1F000290183A784FF138984FF551505C9130707
:10B2000000023306A74033D7C7003314A400598C7B
:10B21000B706F03FC18E014763F429010327C9FF38
:10B22000B397A7003357C700D98F45BFB706F03F84
:10B23000C18E65B7797122D42E84854526D24AD035
:10B24000B2844ECE52CC3A8906D6368AEFF03F828F
:10B25000370710009307F7FFE58FD18093F4F47F51
:10B26000AA89B5E03EC62DC4280022C4EFF05FA530
:10B27000A24621CD324793070002898FB317F7000A
:10B28000D58F3357A70023AAF9003AC6324423AC1E
:10B29000890033348000050423A88900B9C493844D
:10B2A000D4BCAA949307500323209A003385A74067
:10B2B0002320A900B25022544E8592540259F249DB
:10B2C000624A45618280D98F71BF23AAD9007DBFB0
:10B2D0006800EFF0FF9EB24713050502054423AA5C
:10B2E000F900854723A8F90055BF931724001305DB
:10B2F000E5BCCE972320AA00884B1604EFF0FF97F9
:10B30000098C232089007DB779714AD02E892C00C1
:10B3100006D622D426D24ECE52CC2A8AEFF05FE651
:10B32000AA89AE842E844A856C00EFF07FE58327DE
:10B33000090103270A01A2461D8FB24716079D8EF9
:10B34000B307D7006355F002D2072E8633849700E7
:10B350003287A2852A86BA864E85EFA09FA3B25077
:10B36000225492540259F249624A45618280370759
:10B37000F0FFB387E7023386B700D9BF9387F5FFA5
:10B38000184A958785078A07930646010A07AA97F0
:10B39000369763E5E600636AF5008280910603A6AE
:10B3A000C6FF1105232EC5FEEDB71105232E05FEA0
:10B3B000DDB7144993D755401307450163C7F6021B
:10B3C00063DFD700FD8981CD93962700BA9690421E
:10B3D0000545B356B600B395B600631EB6008A079E
:10B3E000BA976366F70001458280B687CDBFF11733
:10B3F0009443E5DA054582803386C502011122CCEB
:10B4000006CEB28532C6EFC0AF922A8409C5324655
:10B410008145EF40FFD62285F2406244056182807B
:10B4200001114AC803A9850022CC52C45AC006CED5
:10B4300026CA4EC656C22E84328B368A63E9260946
:10B44000DE2513F7074851C304408C495848AA8A9F
:10B45000B389B4408D44B384E4020947B3C4E40221
:10B46000138716004E9763F3E400BA8493F70740FE
:10B47000BDCFA6855685EFC0AF8B2A891DE1B147A8
:10B4800023A0FA005E247D5593E707045EA4F240F2
:10B490006244D2444249B249224A924A024B05616F
:10B4A00082800C484E86EFB01FF35E2493F7F7B707
:10B4B00093E707085EA42328240144C84E99B38467
:10B4C00034412320240104C4528963732A01528920
:10B4D00008404A86DA85EF00F0331C440145B38703
:10B4E00027411CC41C403E99232024014DB72686C9
:10B4F0005685EF0090362A895DFD0C485685EFB0E1
:10B50000BFF8B5BFDE25717126D34AD14ECF06D71D
:10B5100022D552CD56CB5AC95EC762C566C393F7D2
:10B520000708AA892E89B284B9C39C49A9E3930567
:10B53000000436C6EFB0DFFF2320A9002328A900AE
:10B54000B24615E1B14723A0F9007D55BA502A54FF
:10B550009A540A59FA496A4ADA4A4A4BBA4B2A4C6F
:10B560009A4C4D61828093070004232AF9009307C7
:10B570000002A30CF1029307000302DA230DF1028B
:10B5800036CE930B5002971A0000938A6A6F054CCF
:10B59000294B26841C2099C363997709B30C9440E6
:10B5A000638E0C00E6862686CA854E85EFF05FE73F
:10B5B000FD576309F518D256E69636DA1C206383E8
:10B5C0000718FD579304140002D002D63ED202D4CD
:10B5D000A301010682DC8C2015465685EFF06FC76B
:10B5E00013841400825721E513F7070109C71307D5
:10B5F0000002A301E10613F7870009C71307B00291
:10B60000A301E10694201307A002638AE602B25761
:10B61000268481462546182093051400130707FD4C
:10B620006372E6068DC63ED61DA00504A5B7330598
:10B6300055413315AC00C98F3ED0A28469BF724713
:10B6400093064700184336CE634707023AD61820C0
:10B650009307E002631DF70418309307A002631BF1
:10B66000F702F2470904138747009C433ACE63C1AF
:10B6700007023ED22DA83307E04093E727003AD6D1
:10B680003ED0F1B7B387670385462E84BA9761B77A
:10B69000FD57C5B7050402D28146814725461820CB
:10B6A00093051400130707FD6376E606F9F20C20F4
:10B6B0000D46171500001305255DEFF08FB911CD6C
:10B6C000971700009387475C1D8D93070004B3977D
:10B6D000A700025505045D8D2AD00C2019461715C8
:10B6E00000001305A55A93041400230CB102EFF0D7
:10B6F0004FB635C197C7FFFF9387470895E70257B5
:10B70000F2471377071009CF91073ECED257D29751
:10B710003EDA41B5B387670385462E84BA9741B7B1
:10B720009D07E19BA107D5B778089706000093868F
:10B7300066CF4A860C104E85EFC00F84FD572A8ACB
:10B74000E316F5FC8357C9007D5593F70704E39F83
:10B7500007DE5255E5BB780897060000938686CC35
:10B760004A860C104E85EFC02FDEC9BF1C46FD1760
:10B770001CC663D90700184E63C5E700A947639349
:10B78000F5007DA61C422E851387170018C28CA3D6
:10B790008280011122CC26CA4AC84EC652C406CEA7
:10B7A0002A89AE893284B304D6007D5A631494008A
:10B7B000014509A80C204E864A85EFF03FFB0504A1
:10B7C000E31645FFF2406244D2444249B249224A5C
:10B7D00005618280357122CD26CB4AC94EC706CF7E
:10B7E00052C556C35AC1DEDEE2DCE6DAAA89AE846F
:10B7F0003289368409C51C4D99E3EFE05F959717B0
:10B800000000938727336399F40C83A44900DE2456
:10B81000A18BEDC79C48FDC393070002A304F1026E
:10B820009307000302D22305F10222C6930B5002B4
:10B83000971A0000938ACA44054C294B4A841C205D
:10B8400099C3639F770DB30C2441638E0C00E68689
:10B850004A86A6854E85EFF0DFF3FD57630FF51C92
:10B860009256E69636D21C206389071CFD571309B1
:10B87000140002C802CE3ECA02CCA309010482D43D
:10B880008345090015465685EFF0AF9C1304190057
:10B89000C24749E913F7070109C713070002A309C3
:10B8A000E10413F7870009C71307B002A309E104F5
:10B8B000834609001307A002638EE606F2474A8416
:10B8C00081462546182093051400130707FD63766B
:10B8D000E60AADCA3ECEBDA0971700009387872722
:10B8E0006395F40083A489001DB797170000938720
:10B8F0006722E39EF4F083A4C90011BFA6854E859C
:10B900002D2E19D97D55FA406A44DA444A49BA497C
:10B910002A4A9A4A0A4BF65B665CD65C0D618280C5
:10B92000050431BF330555413315AC00C98F3EC8FE
:10B930002289B9B7324793064700184336C6634792
:10B9400007023ACE18209307E002631DF70418306F
:10B950009307A002631BF702B2470904138747004D
:10B960009C433AC663C107023ECA2DA83307E04094
:10B9700093E727003ACE3EC8F1B7B3876703854601
:10B980002E84BA9781B7FD57C5B7050402CA814610
:10B9900081472546182093051400130707FD637699
:10B9A000E606F9F20C200D46171500001305C52D0B
:10B9B000EFF02F8A11CD971700009387E72C1D8D8C
:10B9C00093070004B397A700424505045D8D2AC87C
:10B9D0000C201946171500001305452B13091400F8
:10B9E0002304B102EFF0EF8625C197C7FFFF9387CD
:10B9F000E7D895E74247B2471377071009CF910779
:10BA00003EC69257D2973ED215BDB387670385468F
:10BA10002E84BA9741B79D07E19BA107D5B778005F
:10BA200097060000938626D726860C084E85EFB031
:10BA3000BFD4FD572A8AE316F5FCDE2493F70704EA
:10BA4000E39207EC1255C1B5780097060000938683
:10BA500086D426860C084E85EFC00FAFD9BF4111A2
:10BA600022C42E848395E50006C6A12563490500FE
:10BA70007C48AA977CC8B2402244410182805E245F
:10BA80007D777D17F98F5EA4FDB7DE25011122CCED
:10BA900026CA4AC84EC606CE93F70710AA842E843B
:10BAA0003289B68991C78395E50089460146812987
:10BAB0005E247D777D17F98F5EA48315E4006244D0
:10BAC000F240CE864A86B24942492685D244056173
:10BAD00035AA411122C42E848395E50006C60521AE
:10BAE000FD575A24631AF500FD77FD17F98F5EA400
:10BAF000B2402244410182808567D98F5EA468C824
:10BB0000C5BF8395E50015AC15C27D160147B30787
:10BB1000E500B386E5009C2394226396D700630476
:10BB2000C7000507EDF73385D74082800145828045
:10BB3000011122CC26CA4AC806CE4EC6AA842E8936
:10BB4000328409C51C4D99E3EFE06FE097170000C0
:10BB5000938747FE6317F406C0401C4C1CC45E2448
:10BB6000A18BC1C31C48B5CF1C4808409379F90F7D
:10BB70001379F90F1D8D5C486346F500A285268573
:10BB8000192E25E51C440505FD171CC41C40138710
:10BB9000170018C0238037015C486388A7005E2423
:10BBA000858B81CBA9476316F900A2852685E524FC
:10BBB0000DEDF24062444A85D2444249B2490561E2
:10BBC0008280971700009387E7F86314F40080449D
:10BBD00069B7971700009387E7F3E310F4F8C044C0
:10BBE000ADBFA2852685912841D17D59D9B789CD90
:10BBF0009307F00F63F7C7009307A0081CC17D559A
:10BC0000828090A10545828001458280411122C435
:10BC10002A842E85B285368623A401CE06C6EF700F
:10BC2000CF84FD576317F500938781CE9C4391C362
:10BC30001CC0B24022444101828041119387C180DF
:10BC400026C2844322C44AC006C62A892E8491C4CF
:10BC50009C4C81E72685EFE08FCF971700009387F4
:10BC600067ED631BF402C0400317C400931707017C
:10BC7000C18393F68700B5EA93F6070195EEA547D1
:10BC80002320F900136707045AA47D55B2402244CB
:10BC9000924402494101828097170000938787EB05
:10BCA0006314F4008044C9B797170000938787E6B0
:10BCB000E31CF4FAC0444DBF918B85C74C5891C921
:10BCC000930744046385F5004A85EFB0EFFB232A10
:10BCD00004025E242322040093F7B7FD5EA41C48EF
:10BCE0001CC05E2493E787005EA41C4899EB5E2489
:10BCF0001307002093F707286385E700A2854A858C
:10BD000049245E2413F717001DC35C482324040054
:10BD1000B307F0401CCC1C480145ADFB8317C400A1
:10BD200013F7070825D793E707045EA4B9BF898BEB
:10BD3000014791E3584818C4F9BF411122C42A842D
:10BD40002E8523A401CE06C6EF001022FD576317EF
:10BD5000F500938781CE9C4391C31CC0B24022441E
:10BD600041018280DE25011122CC26CA06CE4AC8B6
:10BD70004EC613F78700AA842E8461EFD841634D25
:10BD8000E000B841634AE0000145F2406244D24419
:10BD90004249B2490561828058547DD703A9040005
:10BDA0009396370123A0040063DC060670485E24E6
:10BDB000918B99C75C401D8E5C5899C33C401D8E89
:10BDC0005C540C50814626858297FD575A24631D8A
:10BDD000F5009440F54763E9D706B707402085078B
:10BDE000B3D7D700858BADC31C48232204001CC0E9
:10BDF0009317370163D80700FD576314F5009C4083
:10BE000091E368C84C5823A02401BDDD9307440486
:10BE10006385F5002685EFB02FE7232A0402ADB72E
:10BE20000C500146854626850297FD572A86E31069
:10BE3000F5F89C40ADDF75476385E700594763938C
:10BE4000E70423A0240189B7136707045AA47D558A
:10BE50002DBF83A90501E38909F203A905008D8B94
:10BE600023A0350133093941014791E3D84918C46A
:10BE7000E35C20F11C540C50CA864E8626858297BE
:10BE80006347A0005E2493E707045EA4C9B7AA999C
:10BE90003309A940F1BF9C49ADC3011122CC06CEA4
:10BEA0002A8419C51C4D89E72EC6EFE04FAAB2457A
:10BEB00097170000938707C8639CF5004C40839751
:10BEC000C5009DC722856244F24005616FF09FE97D
:10BED00097170000938707C86394F5000C44C5B713
:10BEE00097170000938707C3E39BF5FC4C44C1BF41
:10BEF000F240624401450561828001458280411122
:10BF000022C42A842E85B285368623A401CE06C695
:10BF1000EF00D007FD576317F500938781CE9C4350
:10BF200091C31CC0B2402244410182801971A6DA3B
:10BF3000AE848395E500A2DC86DE328463DB0500F7
:10BF4000DE2423A0060093F707089DE39307004033
:10BF500015A0300836C66122B246E34305FE72479B
:10BF6000BD67F98F7977BA9793B717009CC2F9BF6D
:10BF7000930700041CC0F6506654D654014509616D
:10BF80008280DE25011122CC06CE26CA4AC8898BC2
:10BF90002E8489CF930774041CC01CC885475CC8D5
:10BFA000F2406244D244424905618280740030000C
:10BFB000AA84EFF0BFF7A2452A892685EFB04FD7B4
:10BFC00019E98317C40013F7072079FBF19B93E766
:10BFD00027005EA4C1B797E7FFFF938767129CD441
:10BFE0005E2408C008C893E707085EA4A2475CC89F
:10BFF000B24799CB8315E4002685392211C55E240A
:10C00000F19B93E717005EA45E243369F9002316C1
:10C01000240179B763F1A504B386C500637DD50219
:10C020009345F6FF8147FD176393F50082803387C0
:10C03000F600034807003387C7002A97230007014B
:10C04000DDB73387F50014233307F500850714A304
:10C05000E319F6FE82808147E5BF81E5B2856FB0C6
:10C060002FCD011122CC06CE26CA4AC84EC6328434
:10C0700001EEEFB06FC10149F24062444A85D244FB
:10C080004249B24905618280AE84AA895520268939
:10C09000E37485FEA2854E85EFB08FC92A8969DDDC
:10C0A000A6852286EFB02FB3A6854E85EFB0CFBD13
:10C0B000E1B7411122C42A842E85B285368623A495
:10C0C00001CE06C6D12DFD576317F500938781CEAB
:10C0D0009C4391C31CC0B240224441018280411163
:10C0E00022C42A842E85B28523A401CE06C65925F2
:10C0F000FD576317F500938781CE9C4391C31CC005
:10C10000B240224441018280411122C42A842E85FA
:10C1100023A401CE06C6AD25FD576317F50093870E
:10C1200081CE9C4391C31CC0B24022444101828015
:10C1300083A7C5FF1385C7FF63D50700AA959C4158
:10C140003E95828013D74501B7071000FD1713D81D
:10C1500046011377F77F9308F07F33FEB700AA8E6E
:10C16000F58FFD81328F1378F87FFD82630B170105
:10C1700005436306180163140701630DFE001A8569
:10C180008280B368AE000543E39B08FEE319E8FE36
:10C19000D18FF5F70543E394EEFF0143E381D5FE2C
:10C1A000054371FF3365AE003333A000C9BF13D719
:10C1B0004501B7071000FD1713D846011377F77F25
:10C1C0009308F07F33F3B7002A8EF58FFD81B28E8E
:10C1D0001378F87FFD8263081703630018030DEBE3
:10C1E000B368A300631408005D8E29CA6385080440
:10C1F0006388D502054595ED8280B3E8C700E380EA
:10C2000008FE795582803365A30065FD630CE80262
:10C21000631408005D8E79DEE39ED5FCE34CE8FCF8
:10C2200063480701E3E867FC6303F302637FF300FD
:10C2300081E57D558280F5DE054582800145E39BE1
:10C2400008FA82805D8E69DA6DBF01458280E3E382
:10C25000CEFB0145E372DEFBE5F1E1BF13D74501FB
:10C26000B7071000FD1713D846011377F77F93081F
:10C27000F07F33FEB700AA8EF58FFD81328F1378E1
:10C28000F87FFD82630E1703630D180129E3B3687D
:10C29000AE00631F08005D8E01EE0143638C08044D
:10C2A00021A8B3E8C7000943639608046DD305A02D
:10C2B000638408046385D50205438DCD7D531DA895
:10C2C000B368AE00094363970802630AE802631487
:10C2D00008005D8E75D2E391D5FEE34FE8FC63491B
:10C2E0000701E3EBC7FD630FFE0001436374FE002B
:10C2F000F1D505431A858280EDFE7D53E5BF5D8E45
:10C3000079DACDBFE36ADFFB0143E3F5EEFFF5F138
:10C3100075B713D74501B7071000FD171347F7FF8F
:10C3200013D84601FD8DF58F931657011378F87FCA
:10C3300099CA1307F07F01456303E8008280D18F1B
:10C340003335F0008280C98D0545E5D5828093D7CD
:10C350004501B70610001387F6FF93F7F77F130622
:10C36000E03F2A886D8F0145FD816354F60099C135
:10C37000828082801306E0417D55E34BF6FE130573
:10C3800030431D8D7D46558F634AA6009387D7BEE7
:10C390003317F7003355A800598D828013053041BB
:10C3A000B307F5403355F7008280935746011317C2
:10C3B000C60093F7F77F797131839386170022D4F3
:10C3C00026D206D64AD02EC83ACA02CE02CC93F65E
:10C3D000E67F2A849354F601B9CA9166938606C013
:10C3E000B69713D645009316C701C607D18E13958D
:10C3F000C5011183C583014878863247C607B70552
:10C400000180C583FD15C2076D8FD98F86071396EE
:10C41000F4018583D18F48C02320040114C45CC477
:10C420002285B2502254925402594561828033656C
:10C43000B700BDE751CD55C33A85EFA0BFF1130753
:10C4400015031378F7011587631D080A1008931662
:10C450002700B306D6408A8813182700CC46B38736
:10C460000601F116CCC7E39BD8FE7D170A07329769
:10C47000232007009306C7FF6309E60036872320C1
:10C4800007009306C7FFE31BE6FE91679387C7C0CB
:10C49000898FC60742485245E246B886C583A9BF80
:10C4A00015C1A167135547009316C7013367F500FF
:10C4B00013D645004207D18E1395C5014183FD1760
:10C4C00001481DBFA1678146FD17014701482DB7EF
:10C4D000814681470147014805B72E852E89EFA087
:10C4E0007FE7130715051378F70113050502158774
:10C4F000E30E08F489476306F70009471008B148BE
:10C5000035A8B306E0408A061008B106130E0002F3
:10C51000B29693182700330E0E4183A5C6FF9C42A6
:10C5200033831601B3D5C501B3970701DD8D2320F1
:10C53000B300F116E313D6FE42497D171C10BE98D6
:10C540003319090123A828FF15B70328C50018418E
:10C5500054410C4521659307F5FF13560801139EBE
:10C5600035007D8E9358D70193D7D6011313080158
:10C570008E064111B3E7C701B3E616011353030159
:10C58000131E3700930816007915F5810E033EC47B
:10C5900036C272C033F5A8001358F801B3E5650040
:10C5A00005C97177130707403A961307E07F635D6B
:10C5B000C7041306F07F01478147320752063183D3
:10C5C0007E08518F336707013E85BA85410182801D
:10C5D000D58FCD8FB3E7C70105E2F1CB81479546F3
:10C5E00093D53600139797009396D701B3E7B6001B
:10C5F00031831376F67FD1B7CDDF01481306F07F84
:10C6000037070800814755BF6346C00A9307C0FC3F
:10C61000634FF60E9307D0033386C74093575640B7
:10C6200037070800D98D139527000A8781462EC643
:10C63000B308A10011077D8AB3E6C601630917019B
:10C64000032E07001107B3E6C601E31B17FF0D47D2
:10C650001D8F79CA93080101AA9883A808FF130EB9
:10C660000002330ECE40B398C801B3E6160175CB75
:10C670000A070A95B30EE1008A880C41032345009E
:10C680009108B3D5C5003313C301B3E5650023AEEC
:10C69000B8FE1105E3931EFF9145B387F540B245FF
:10C6A00008082A97B3D5C5002328B7FE61A801461C
:10C6B000014721B713974600139547003367C70119
:10C6C000F182F18392053337E000C98ECD8FD98E88
:10C6D00013F7760011C713F7F6009145631CB702F4
:10C6E000370780007D8FE30D07EE05061307F07F07
:10C6F000E301E6EC370780FF7D177D8F9317D701A5
:10C700008D8226071376F67FD58F31837DB58546DA
:10C710008147014613B7C6FF13471700BA9737077B
:10C72000800091067D8FC1B78A85B388A50083A854
:10C7300008009105050623AE15FFE358C7FE114713
:10C74000B307F7408A078A97180823A007009107C4
:10C75000E39DE7FE0247B336D0009247D98E0146EB
:10C7600085BF854701472DBF9307800523A4F1CEE0
:10C770007D5582809307800523A4F1CE7D5582806C
:10C780009307800523A4F1CE01458280930780059D
:10C7900023A4F1CE7D5582809307800523A4F1CE9A
:10C7A0007D55828000000000000000000000B040C5
:10C7B0006666666666660A400000803F00000040CC
:10C7C0000000304172656400677265656E000000AC
:10C7D000626C7565000000006C65645F6D3100007F
:10C7E0006C65645F6D3200006C65645F6D330000E2
:10C7F0006C65645F6D3400006B6579733A25642C59
:10C8000025642C25642C2564096164633A25342E43
:10C8100034662C25342E34662C25342E34662C2593
:10C82000342E346609207469636B3A25750A00005A
:10C83000FA5100004C520000A052000000530000CA
:10C8400040530000765300008C97FFFF1096FFFFC7
:10C850002097FFFF2897FFFF2097FFFF4096FFFFDD
:10C860002097FFFF2897FFFF1096FFFF1096FFFF0E
:10C870004096FFFF2897FFFF8297FFFF8297FFFFF9
:10C880008297FFFF4096FFFFCE9CFFFFC09BFFFFFC
:10C89000C09BFFFFBE9BFFFFC69BFFFFC69BFFFF2A
:10C8A0008C9BFFFFBE9BFFFFC69BFFFF8C9BFFFF88
:10C8B000C69BFFFFBE9BFFFFBA9CFFFFBA9CFFFF1A
:10C8C000BA9CFFFF8C9BFFFF0001020203030303DE
:10C8D0000404040404040404050505050505050510
:10C8E00005050505050505050606060606060606F0
:10C8F00006060606060606060606060606060606D8
:10C9000006060606060606060707070707070707BF
:10C9100007070707070707070707070707070707A7
:10C920000707070707070707070707070707070797
:10C930000707070707070707070707070707070787
:10C94000070707070707070708080808080808086F
:10C950000808080808080808080808080808080857
:10C960000808080808080808080808080808080847
:10C970000808080808080808080808080808080837
:10C980000808080808080808080808080808080827
:10C990000808080808080808080808080808080817
:10C9A0000808080808080808080808080808080807
:10C9B00008080808080808080808080808080808F7
:10C9C0000808080808080808FFFFFFFFFFFFEF7FBF
:10C9D000494E4600696E66004E414E006E616E0023
:10C9E0003000000030313233343536373839414287
:10C9F0004344454600000000303132333435363789
:10CA000038396162636465660000000065256C6406
:10CA1000000000000000C07FBABCFFFFA6BCFFFF03
:10CA2000D8BCFFFFDEBCFFFFBABCFFFF0000000068
:10CA3000000000000000E03F000000000000F03FA8
:10CA400000000000000000400000C0FFFFFFDF41C9
:10CA50009535A094FFFFDF3F35E5AF350000E03F9F
:10CA60009535A094FFFFCF3F6E660000696E697434
:10CA700079000000616E000035000000CEFBFFFF72
:10CA8000CB030000010000000000000034000000A3
:10CA9000CEFBFFFFCB030000010000000000000000
:10CAA000BC89D897B2D29C3C33A7A8D523F6493984
:10CAB0003DA7F444FD0FA5329D978CCF08BA5B25A6
:10CAC000436FAC6428066811000000000000F83FC6
:10CAD00061436F63A787D23FB3C8608B288AC63F84
:10CAE000FB799F501344D33F000000000000244016
:10CAF0000000000000001C40000000000000144086
:10CB0000496E66696E697479000000004E614E00DE
:10CB10000000000000000000000000000000000015
:10CB20000000000000000000000000000000000005
:10CB300000000000000000000000000000000000F5
:10CB400000000000000000000000000000000000E5
:10CB500000000000000000000000000000000000D5
:10CB600000000000000000000000000000000000C5
:10CB700043000000504F5349580000002E000000B1
:10CB80000080E03779C34143176E05B5B5B89346C9
:10CB9000F5F93FE9034F384D321D30F94877825A95
:10CBA0003CBF737FDD4F1575000000000000F03FB3
:10CBB0000000000000002440000000000000594078
:10CBC0000000000000408F40000000000088C340CB
:10CBD00000000000006AF8400000000080842E4140
:10CBE00000000000D01263410000000084D797418C
:10CBF0000000000065CDCD41000000205FA0024292
:10CC0000000000E876483742000000A2941A6D4206
:10CC1000000040E59C30A2420000901EC4BCD642F9
:10CC200000003426F56B0C430080E03779C34143A4
:10CC300000A0D8855734764300C84E676DC1AB431A
:10CC4000003D9160E458E143408CB5781DAF154438
:10CC500050EFE2D6E41A4B4492D54D06CFF0804413
:10CC6000F64AE1C7022DB544B49DD9794378EA4428
:10CC700005000000190000007D000000232D302B6E
:10CC800020000000686C4C00656667454647000060
:10CC9000002020202020202020202828282828208C
:10CCA0002020202020202020202020202020202084
:10CCB00020881010101010101010101010101010EC
:10CCC00010040404040404040404041010101010DC
:10CCD00010104141414141410101010101010101A6
:10CCE00001010101010101010101010110101010F8
:10CCF0001010424242424242020202020202020278
:10CD000002020202020202020202020210101010CB
:10CD100020000000000000000000000000000000F3
:10CD20000000000000000000000000000000000003
:10CD300000000000000000000000000000000000F3
:10CD400000000000000000000000000000000000E3
:10CD500000000000000000000000000000000000D3
:10CD600000000000000000000000000000000000C3
:10CD700000000000000000000000000000000000B3
:10CD800000000000000000000000000000000000A3
:04CD9000000000009F
:10CD9400000000000102030401020304060708095D
:10CDA4000000000030CB000050CB000010CB00008E
:10CDB400000000000000000000000000000000006F
:10CDC400000000000000000000000000000000005F
:10CDD400000000000000000000000000000000004F
:10CDE400000000000000000000000000000000003F
:10CDF400000000000000000000000000000000002F
:10CE040043000000000000000000000000000000DB
:10CE1400000000000000000000000000000000000E
:10CE240043000000000000000000000000000000BB
:10CE340000000000000000000000000000000000EE
:10CE4400430000000000000000000000000000009B
:10CE540000000000000000000000000000000000CE
:10CE6400430000000000000000000000000000007B
:10CE740000000000000000000000000000000000AE
:10CE8400430000000000000000000000000000005B
:10CE9400000000000000000000000000000000008E
:10CEA400430000000000000000000000000000003B
:10CEB400000000000000000000000000000000006E
:10CEC400430000000000000000000000000000001B
:10CED400000000000000000000000000000000004E
:10CEE400EEBB000020AA00000000000090CC00006F
:10CEF4007CCB0000F4C90000F4C90000F4C90000B0
:10CF0400F4C90000F4C90000F4C90000F4C9000029
:10CF1400F4C90000F4C90000FFFFFFFFFFFFFFFF9B
:10CF2400FFFFFFFFFFFF0000010041534349490099
:10CF340000000000000000000000000000000000ED
:10CF44000000000000000000000041534349490074
:10CF540000000000000000000000000000000000CD
:10CF640000000000000000000000000000000000BD
:10CF740000D8B80502040608CC06002010000020E2
:08CF8400100000200000000075
:00000001FF
